:100000000C9419140C944A140C944A140C944A1429
:100010000C944A140C944A140C944A140C944A14E8
:100020000C944A140C944A140C944A140C944A14D8
:100030000C944A140C944A140C944A140C944A14C8
:100040000C944A140C944A140C944A140C944A14B8
:100050000C944A140C944A140C944A140C94141ED4
:100060000C944A140C94F1230C94C8230C944A1455
:100070000C944A140C944A140C944A140C944A1488
:100080000C944A140C944A140C944A140C944A1478
:100090000C944A140C944A140C944A140C944A1468
:1000A0000C944A140C944A140C944A140C944A1458
:1000B0000C944A140C944A140C944A140C944A1448
:1000C0000C944A140C944A140C944A140C944A1438
:1000D0000C944A140C944A140C944A140C944A1428
:1000E0000C944A14EB26EE26DD26E126E52625278C
:1000F000F226F626FC26002704270A270E271227B9
:10010000252718271C2720270000000000000000DA
:1001100000000000000000000000000000000000DF
:1001200000000000000000000000000000000000CF
:1001300000000000000000000000000000000000BF
:1001400000000000000000000000000000000000AF
:10015000000000000000000000000000000000009F
:10016000000000000000000000000000010000008E
:10017000000000000000000000000000000000007F
:10018000000000000000000000000000000000006F
:10019000000000000100000000000000000000005E
:1001A000000000000000000000000000000000004F
:1001B0000000000000000000000000C0030000007C
:1001C000000000000000000000000000000000002F
:1001D000000000000000000000000000000000001F
:1001E000000000A007000000000000000000000068
:1001F00000000000000000000000000000000000FF
:100200000000000000000000000000E00B00000003
:1002100000000000000000000000000000000000DE
:1002200000000000000000000000000000000000CE
:10023000000000E00F0000000000000000000000CF
:1002400000000000000000000000000000000000AE
:100250000000000000000000000000F80F00000097
:10026000000000000000000000000000000000008E
:10027000000000000000000000000000000000007E
:10028000000000F03F00000000000000000000003F
:10029000000000000000000000000000000000005E
:1002A0000000000000000000000000FC3F00000013
:1002B000000000000000000000000000000000003E
:1002C000000000000000000000000000000000002E
:1002D000000000FD7F0000000000000000000000A2
:1002E000000000000000000000000000000000000E
:1002F0000000000000000000000000FE7F00000081
:1003000000000000000000000000000000000000ED
:1003100000000000000000000000000000000000DD
:10032000000000FFFF0100000000000000000000CE
:1003300000000000000000000000000000000000BD
:100340000000000000000000000080FFFF0200002D
:10035000000000000000000000000000000000009D
:10036000000000000000000000000000000000008D
:10037000000080FFFF0300000000000000000000FC
:10038000000000000000000000000000000000006D
:1003900000000000000000000000E0FFFF0300007C
:1003A000000000000000000000000000000000004D
:1003B000000000000000000000000000000000003D
:1003C0000000C0FFFF070000000000000000000068
:1003D000000000000000000000000000000000001D
:1003E00000000000000000000000F0FFFF0F000010
:1003F00000000000000000000000000000000000FD
:1004000000000000000000000000000000000000EC
:100410000000F0FFFF1F00000000000000000000CF
:1004200000000000000000000000000000000000CC
:1004300000000000000000000000F8FFFF1F0000A7
:1004400000000000000000000000000000000000AC
:10045000000000000000000000000000000000009C
:100460000000F8FFFF3F0000000000000000000057
:10047000000000000000000000000000000000007C
:1004800000000000000000000000FEFFFF3F000031
:10049000000000000000000000000000000000005C
:1004A000000000000000000000000000000000004C
:1004B0000000FCFFFFFF0000000000000000000043
:1004C000000000000000000000000000000000002C
:1004D00000000000000000000000FFFFFF7F0000A0
:1004E000000000000000000000000000000000000C
:1004F00000000000000000000000000000000000FC
:100500000000FFFFFFFF01000000000000000000EE
:1005100000000000000000000000000000000000DB
:1005200000000000000000000080FFFFFFFF02004D
:1005300000000000000000000000000000000000BB
:1005400000000000000000000000000000000000AB
:100550000080FFFFFFFF030000000000000000001C
:10056000000000000000000000000000000000008B
:10057000000000000000000000A0FFFFFFFF0500DA
:10058000000000000000000000000000000000006B
:10059000000000000000000000000000000000005B
:1005A00000E0FFFFFFFF0700000000000000000068
:1005B000000000000000000000000000000000003B
:1005C000000000000000000000E0FFFFFFFF070048
:1005D000000000000000000000000000000000001B
:1005E000000000000000000000000000000000000B
:1005F00000E0FFFFFFFF0F00000000000000000010
:1006000000000000000000000000000000000000EA
:10061000000000000000000000F8FFFFFEFF1F00C8
:1006200000000000000000000000000000000000CA
:1006300000000000000000000000000000000000BA
:1006400000F0FF7FFDFF1F00000000000000000021
:10065000000000000000000000000000000000009A
:10066000000000000000000000FCFF3FFCFF3F0016
:10067000000000000000000000000000000000007A
:10068000000000000000000000000000000000006A
:1006900000FCFF5FF8FF3F000000000000000000CA
:1006A000000000000000000000000000000000004A
:1006B000000000000000000000FCFF1FF4FF7F00AE
:1006C000000000000000000000000000000000002A
:1006D000000000000000000000000000000000001A
:1006E00000FEFF1FF0FFFF00000000000000000000
:1006F00000000000000000000000000000000000FA
:10070000000000000000000000FFFF07F0FF7F0076
:1007100000000000000000000000000000000000D9
:1007200000000000000000000000000000000000C9
:1007300000FEFF0FE0FFFF010000000000000000CE
:1007400000000000000000000000000000000000A9
:10075000000000000000000080FFFF07C0FFFF0056
:100760000000000000000000000000000000000089
:100770000000000000000000000000000000000079
:1007800080FFFF03C0FFFF03000000000000000027
:100790000000000000000000000000000000000059
:1007A0000000000000000000C0FFFF0180FFFF010B
:1007B0000000000000000000000000000000000039
:1007C0000000000000000000000000000000000029
:1007D00080FFFF0300FFFF07000000000000000093
:1007E0000000000000000000000000000000000009
:1007F0000000000000000000E0FFFF0080FFFF039A
:1008000000000000000000000000000000000000E8
:100810000000000000000000C00000000000000018
:10082000E0FFFF0000FEFF07000000000000800660
:1008300000000000000000000000000000000000B8
:10084000E003000000000000E0FF7F0100FFFF0F59
:10085000000000000000A0030000000000000000F5
:100860000000000000000000C02F00000000000099
:10087000E8FF7F0000FCFF0F000000000000E80719
:100880000000000000000000000000000000000068
:10089000C0BF000000000000F0FF3F0000FEFF1F8F
:1008A000000000000000FF03000000000000000046
:1008B0000000000000000000C0FF05000000000074
:1008C000F8FF7F0000F8FF1F0000000000A0FE07F7
:1008D0000000000000000000000000000000000018
:1008E000E0FF170000000000F8FF1F0000FCFF1FE2
:1008F0000000000000E8FF0300000000000000000E
:100900000000000000000000C0FF7F0000000000A9
:10091000F8FF1F0000F0FF3F0000000000FAFF0793
:1009200000000000000000000000000000000000C7
:10093000E0FFFF0100000000FCFF0F0000F8FF3F98
:100940000000000080FFFF07000000000000000022
:100950000000000000000000C0FFFF0B00000000CE
:10096000FCFF1F0000E0FF7F0000000050FFFF07BA
:100970000000000000000000000000000000000077
:10098000E0FFFF2F00000000FEFF070000F0FF7FE8
:1009900000000000F4FFFF0700000000000000005E
:1009A0000000000000000000E0FFFFBF00000000AA
:1009B000FEFF070000E0FFFF00000000FCFFFF0F4C
:1009C0000000000000000000000000000000000027
:1009D000E0FFFFFF02000000FFFF070000C0FF7FF5
:1009E000000000C0FFFFFF07000000000000000043
:1009F0000000000000000000E0FFFFFF0700000013
:100A0000FEFF070000C0FFFF00000090FFFFFF0F88
:100A100000000000000000000000000000000000D6
:100A2000E0FFFFFF1F000080FFFF010000C0FFFF8D
:100A3000010000E8FFFFFF070000000000000000C9
:100A40000000000000000000E0FFFFFF7F0000004A
:100A5000FFFF03000080FFFF010000FCFFFFFF0F0E
:100A60000000000000000000000000000000000086
:100A7000F0FFFFFFFF000080FFFF01000080FFFF8D
:100A8000020080FFFFFFFF070000000000000000E1
:100A90000000000000000000E0FFFFFFFF050080F5
:100AA000FFFF01000000FFFF010040FFFFFFFF0FFD
:100AB0000000000000000000000000000000000036
:100AC000E0FFFFFFFF0700C0FFFF00000080FFFF07
:100AD0000300F0FFFFFFFF07000000000000000020
:100AE0000000000000000000E0FFFFFFFF3F00806B
:100AF000FFFF01000000FEFF0300E8FFFFFFFF0F04
:100B000000000000000000000000000000000000E5
:100B1000F0FFFFFFFF5F00E0FF7F00000000FFFF2E
:100B20000700FEFFFFFFFF070000000000000000BD
:100B30000000000000000000E0FFFFFFFFFF01C019
:100B4000FFFF00000000FEFF0700FDFFFFFFFF0F9B
:100B50000000000000000000000000000000000095
:100B6000F0FFFFFFFFFF02E0FF7F00000000FEFF3D
:100B700003C0FFFFFFFFFF070000000000000000B0
:100B80000000000000000000E0FFFFFFFFFF07E0A3
:100B9000FF7F00000000FCFF0FC0FFFFFFFFFF0F03
:100BA0000000000000000000000000000000000045
:100BB000F0FFFFFFFFFF0FE0FF3F00000000FCFF22
:100BC00007F8FFFFFFFFFF0F00000000000000001C
:100BD0000000000000000000E0FFFFFFFFFF3FE01B
:100BE000FF3F00000000FCFF0FF8FFFFFFFFFF0FBB
:100BF00000000000000000000000000000000000F5
:100C0000F0FFBFFFFFFF7FF0FF3F00000000F8FF95
:100C10000FFDFFFFFFFDFF070000000000000000C8
:100C20000000000000000000E0FF3FFDFFFFFFF1BB
:100C3000FF3F00000000F8FF1FFFFFFFBFF8FF0F9E
:100C400000000000000000000000000000000000A4
:100C5000F0FF1FF4FFFFFFF5FF1F00000000F4FF8F
:100C6000AFFFFFFF1FFCFF0F0000000000000000AF
:100C70000000000000000000E0FF3FE0FFFFFFFF7A
:100C8000FF1F00000000F8FFFFFFFFFF2BF8FF0F22
:100C90000000000000000000000000000000000054
:100CA000F0FF1F80FFFFFFFFFF0F00000000F0FFBD
:100CB000FFFFFFFF05F8FF07000000000000000035
:100CC0000000000000000000E0FF3F00FEFFFFFF0B
:100CD000FF1F00000000F0FFFFFFFF7F01F8FF0F84
:100CE0000000000000000000000000000000000004
:100CF000F0FF1F00FDFFFFFFFF0F00000000E8FFF7
:100D0000FFFFFF3F00FCFF070000000000000000A5
:100D10000000000000000000E0FF3F00F0FFFFFFC8
:100D2000FF1F00000000F0FFFFFFFF2F00F8FF0F84
:100D300000000000000000000000000000000000B3
:100D4000F0FF5F00E0FFFFFFFF0700000000E0FF93
:100D5000FFFFFF0700F8FF07000000000000000091
:100D60000000000000000000E0FF3F0080FFFFFFE8
:100D7000FF0F00000000E0FFFFFFFF0500F8FF0F7E
:100D80000000000000000000000000000000000063
:100D9000F0FF1F0000FFFFFFFF0700000000F0FF53
:100DA000FFFFFF0000FCFF07000000000000000044
:100DB0000000000000000000E0FF3F0000FCFFFF1B
:100DC000FF0F00000000E0FFFFFFBF0000F8FF0F73
:100DD0000000000000000000000000000000000013
:100DE000E0FF3F0000F4FFFFFF0700000000E0FF0E
:100DF000FFFF1F0000FCFF070000000000000000D4
:100E00000000000000000000E0FF7F0000F0FFFF96
:100E1000FF0700000000C0FFFFFF170000F8FF0FF2
:100E200000000000000000000000000000000000C2
:100E3000E0FF3F0000C0FFFFFF0700000000E0FFF1
:100E4000FFFF070000FEFF07000000000000000099
:100E50000000000000000000C0FF3F000080FFFF16
:100E6000FF0700000000C0FFFFFF050000FCFF07B8
:100E70000000000000000000000000000000000072
:100E8000F0FF7F000080FEFFFF0300000000C0FFB6
:100E9000FFFF000000FCFF07000000000000000052
:100EA0000000000000000000C0FF3F000000FEFF47
:100EB000FF0700000000C0FFFFBF000000FCFF07AD
:100EC0000000000000000000000000000000000022
:100ED000E0FF7F000000FCFFFF0300000000C0FFF8
:100EE000FF3F000000FEFF070000000000000000C0
:100EF0000000000000000000C0FF7F000000F0FFC5
:100F0000FF0300000000C0FFFF3F000000FCFF07E0
:100F100000000000000000000000000000000000D1
:100F2000C0FF3F000000E8FFFF0300000000C0FF1B
:100F3000FF07000000FEFF030000000000000000AB
:100F40000000000000000000C0FF7F000000C0FFA4
:100F5000FF0300000000C0FFFF0F000000FCFF07C0
:100F60000000000000000000000000000000000081
:100F7000C0FF7F000000A0FFFF0300000000C0FFD3
:100F8000FF01000000FEFF03000000000000000061
:100F90000000000000000000C0FFFF00000040FF54
:100FA000FF030000000080FFFF03000000FEFF03BE
:100FB0000000000000000000000000000000000031
:100FC000C0FF7F00000000FFFF0300000000C0FF23
:100FD000FF00000000FDFF03000000000000000013
:100FE000000000000000000080FFFF00000000FE85
:100FF000FF030000000080FFFF00000000FFFF0370
:1010000000000000000000000000000000000000E0
:10101000C0FFFF00000000FFFF0300000000C0FF52
:101020007F00000000FEFF03000000000000000041
:10103000000000000000000080FFFF00000000FE34
:10104000FF030000000080FFFF00000000FFFF0220
:101050000000000000000000000000000000000090
:1010600080FFFF00000000FEFF0300000000C0FF43
:101070007F00000000FFFF010000000000000000F2
:10108000000000000000000080FFFF01000000FEE3
:10109000FF030000000080FFFF00000000FFFF01D1
:1010A0000000000000000000000000000000000040
:1010B00000FFFF01000000FDFF0300000000C0FF73
:1010C0007F00000080FFFF01000000000000000022
:1010D000000000008008000000FFFF01000000FE8B
:1010E000FF030000000080FFFF00000000FFFF0181
:1010F0000000400400000000000020B57FF755020A
:1011000080FFFF01000000FFFF0300000000C0FFA0
:101110007F00000080FFFF0040EADFFB5502000077
:101120000080EEFFFFFFFFBF00FFFF03000000FE97
:10113000FF030000000080FFFF00000080FFFF01B0
:10114000ED7FFFFFFFBF020040FFFFFFFFFFFFEF4C
:101150009FFEFF03000000FEFF0300000000C0FF31
:101160007F000000C0FFFFFAFFFFFFFFFFFF7F01CE
:101170005DFDFFFFFFFFFFFFFFFFFF03000000FE1D
:10118000FF030000000080FFFF000000C0FFFFF72A
:10119000FFFFFFFFFFFFFF7FFEFFFFFFFFFFFFFFE0
:1011A000FFFFFF07000000FEFF0300000000C0FF7C
:1011B0007F000000C0FFFFFFFFFFFFFFFFFFFFBF3B
:1011C000FCFFFFFFFFFFFFFFFFFFFF07000000FC2A
:1011D000FF0300000000C0FFFF000000C0FFFFFF92
:1011E000FFFFFFFFFFFFFF7FFCFFFFFFFFFFFFFF92
:1011F000FFFFFF07000000FEFF0300000000C0FF2C
:101200003F000000F0FFFFFFFFFFFFFFFFFFFF1F9A
:10121000F8FFFFFFFFFFFFFFFFFFFF0F000000FED3
:10122000FF0700000000C0FF7F000000E0FFFFFF9D
:10123000FFFFFFFFFFFFFF3FF8FFFFFFFFFFFFFF85
:10124000FFFFFF07000000FCFF0300000000C0FFDD
:101250007F000000F0FFFFFFFFFFFFFFFFFFFF1F0A
:10126000F0FFFFFFFFFFFFFFFFFFFF3F000000FE5B
:10127000FF0700000000C0FF7F000000F0FFFFFF3D
:10128000FFFFFFFFFFFFFF1FF0FFFFFFFFFFFFFF5D
:10129000FFFFFF5F000000FCFF0300000000E0FF15
:1012A0003F000000FFFFFFFFFFFFFFFFFFFFFF0FFB
:1012B000E0FFFFFFFFFFFFFFFFFFFFFF030000FC5A
:1012C000FF0700000000C0FF7F000080FEFFFFFF5F
:1012D000FFFFFFFFFFFFFF0FF0FFFFFFFFFFFFFF1D
:1012E000FFFFFFFF070000FEFF0700000000E0FF18
:1012F0003F0000F0FFFFFFFFFFFFFFFFFFFFFF07C3
:10130000C0FFFFFFFFFFFFFFFFFFFFFF3F0000FCED
:10131000FF0F00000000C0FF7F0000F4FFFFFFFF91
:10132000FFFFFFFFFFFFFF0FE0FFFFFFFFFFFFFFDC
:10133000FFFFFFFF7F0000FCFF0700000000F0FF41
:101340003F0000FFFFFFFFFFFFFFFFFFFFFFFF0367
:1013500080FFFFFFFFFFFFFFFFFFFFFFFF0300F81E
:10136000FF0F00000000E0FF3F0080FEFFFFFFFFD7
:10137000FFFFFFFFFFFFFF0380FFFFFFFFFFFFFFF8
:10138000FFFFFFFFFF0B00FCFF0700000000E0FF76
:101390003F00F0FFFFFFFFFFFFFFFFFFFFFFFF0129
:1013A00000FFFF97000050FDFFFFFFFFFF1F00F849
:1013B000FF0F00000000E0FF3F00E0FFFFFFFFFF26
:1013C000FF4A0000F2FFFF0180FFFF0F0080005284
:1013D000FFFFFFFFFF3F00FCFF0F00000000F8FFD2
:1013E0001F00FEFFFFFFFFFF0A000000E0FFFF00FD
:1013F00000FEFF0F00000000E8FFFFFFFFFF01F805
:10140000FF1F00000000F0FF3F00FEFFFFFFFF97FF
:1014100000000000E0FFFF0100FFFF0F00000000E0
:1014200000FFFFFFFFFF02F8FF0F00000000F0FFCA
:101430001FC0FFFFFFFF7F0100000000F8FF7F00DB
:1014400000FCFF1F0000000000E8FFFFFFFF07F0A7
:10145000FF1F00000000F0FF1FC0FFFFFFFF2F0075
:1014600000000000F0FF7F0000FEFF3F00000000D2
:1014700000A0FFFFFFFF1FF8FF1F00000000F8FFA4
:101480001FF8FFFFFFFF020000000000F8FF3F0011
:1014900000F8FF3F000000000000FAFFFFFF3FF0F0
:1014A000FF3F00000000F8FF1FF8FFFFFFBF000034
:1014B00000000000FAFF3F0000F8FFBF000000003E
:1014C0000000F0FFFFFF7FF0FF1F00000000F4FFAF
:1014D0000FFFFFFFFF07000000000000FCFF1F00E0
:1014E00000F0FF7F00000000000000FFFFFFFFF1A1
:1014F000FF3F00000000FCFF1FFEFFFFFF09000090
:1015000000000000FEFF3F0000E8FFFF00000000B9
:10151000000080FCFFFFFFF3FF3F00000000FCFF26
:10152000E7FFFFFF3F00000000000000FFFF0F008B
:1015300000E0FFFF01000000000000F0FFFFFFEFF0
:10154000FF7F00000000FCFFDFFFFFFF57000000EF
:1015500000000000FEFF0F0000D0FFFF00000000B1
:10156000000000A0FFFFFFFFFF3F00000000FCFFA6
:10157000FFFFFFFF0B00000000000080FFFF0300E3
:1015800000C0FFFF0300000000000040FFFFFFFF5E
:10159000FF7F00000000FDFFFFFFFFFF02000000D3
:1015A00000000080FFFF070000C0FFFF03000000F5
:1015B00000000000FEFFFFFFFF7F00000000FEFFB5
:1015C000FFFFFFBF00000000000000E0FFFF03007E
:1015D0000080FFFF0700000000000000F0FFFFFF99
:1015E000FFFF00000000FEFFFFFFFF2F00000000D4
:1015F000000000C0FFFF03000000FFFF0F0000001D
:1016000000000000E8FFFFFFFFFF00000000FFFFF9
:10161000FFFFFF1700000000000000F0FFFF0000C8
:101620000000FFFF1F0000000000000080FFFFFF20
:10163000FFFF01000000FFFFFFFFFF0300000000AD
:10164000000000E0FFFF01000000FEFF0F000000AF
:101650000000000040FFFFFFFFFF00000000FFFF51
:10166000FFFFFF0000000000000000F8FF7F000007
:101670000000FCFF3F0000000000000000FCFFFF36
:10168000FFFF01000040FFFFFFFFBF000000000060
:10169000000000F8FF7F00000000FEFF3F00000098
:1016A0000000000000FAFFFFFFFF03000080FFFFC3
:1016B000FFFF1F0000000000000000FEFF3F0000D1
:1016C0000000F8FFFF0000000000000000E0FFFF46
:1016D000FFFF03000080FFFFFFFF2F00000000005E
:1016E000000000FCFF7F00000000F8FF7F0000000A
:1016F0000000000000D0FFFFFFFF050000C0FFFF5B
:10170000FFFF030000000000000000FFFF0F0000CB
:101710000000F0FFFF010000000000000080FFFF5C
:10172000FFFF070000C0FFFFFFFF050000000000F3
:10173000000000FFFF1F00000000E0FFFF010000AD
:10174000000000000000FFFFFFFF030000E0FFFFBC
:10175000FFFF0000000000000000C0FFFF070000C6
:101760000000E0FFFF070000000000000000FCFF99
:10177000FFFF0F0000E0FFFFFFBF000000000000C0
:10178000000080FFFF0F00000000C0FFFF0B000003
:10179000000000000000FAFFFFFF070000F0FFFF5D
:1017A000FF3F0000000000000000E0FFFF0300001A
:1017B000000080FFFF0F0000000000000000F0FFAD
:1017C000FFFF1F0000E0FFFFFF1F00000000000000
:1017D0000000E8FFFF030000000080FFFF2F000073
:1017E000000000000000D0FFFFFF0F0000F8FFFF27
:1017F000FF070000000000000000F0FFFF010000F4
:10180000000000FFFF3F0000000000000000C0FFDC
:10181000FFFF1F0000F0FFFFFF07000000000000B7
:101820000000F8FF7F010000000000FEFF5F0000E5
:1018300000000000000080FFFFFF3F0000FCFFFFF2
:10184000FF010000000000000000FEFFFF0000009C
:10185000000000FCFFFF000000000000000000FF8F
:10186000FFFF3F0000F8FFFF7F01000000000000C5
:101870000000FEFF7F000000000000FAFF7F010073
:1018800000000000000000FEFFFF3F0000FEFFFF21
:101890007F000000000000000080FEFF1F0000002D
:1018A000000000F8FFFF010000000000000000FC45
:1018B000FFFF7F0000FCFFFFBF00000000000000F2
:1018C0000080FFFF3F000000000000F0FFFF03006A
:1018D00000000000000000F8FFFF7F0000FEFFFF97
:1018E0001F0000000000000000C0FFFF0F0000000C
:1018F000000000E0FFFF0F0000000000000000F00B
:10190000FFFFFF0000FFFFFF1F00000000000000BE
:1019100000D0FFFF0F000000000000E0FFFF1700F5
:1019200000000000000000E0FFFFFF0000FFFFFFDD
:10193000070000000000000000F0FFFF07000000AB
:1019400000000080FFFF1F0000000000000000C03A
:10195000FFFFFF0100FFFFFF070000000000000085
:1019600000F4FFFF05000000000000C0FFFF3F0083
:1019700000000000000000C0FFFFFF01C0FFFFFFEC
:10198000010000000000000000FCFFFF010000005B
:1019900000000000FFFFFF0000000000000000004A
:1019A000FFFFFF0380FFFFFF0300000000000000B7
:1019B00000FEFFFF0100000000000000FEFFFF002E
:1019C0000000000000000000FFFFFF07E0FFFF7FB6
:1019D000000000000000000080FFFF7F000000000A
:1019E00000000000FCFFFF030000000000000000FA
:1019F000FCFFFF07C0FFFF7F0000000000000000A9
:101A000040FFFF7F0000000000000000FCFFFF0718
:101A10000000000000000000FEFFFF07E0FFFF3FA6
:101A20000000000000000000E0FFFF1F00000000B9
:101A300000000000F0FFFF1F000000000000000099
:101A4000F8FFFF0FF0FFFF3F000000000000000064
:101A5000E8FFFF3F0000000000000000F0FFFF2F44
:101A60000000000000000000F0FFFF1FE8FFFF0F74
:101A70000000000000000000F8FFFF070000000069
:101A800000000000C0FFFF7F000000000000000019
:101A9000E0FFFF1FF8FFFF1700000000000000003C
:101AA000FDFFFF0F0000000000000000A0FFFFFF8F
:101AB0000000000000000000D0FFFF3FFCFFFF0718
:101AC0000000000000000000FFFFFF010000000018
:101AD0000000000000FFFFFF030000000000000006
:101AE000C0FFFF7FF8FFFF0500000000000000407E
:101AF000FFFFFF03000000000000000080FEFFFF6A
:101B0000070000000000000080FFFF3FFDFFFF0313
:101B100000000000000000E0FFFF7F000000000068
:101B20000000000000FCFFFF1F000000000000009C
:101B300000FFFF7FFFFFFF0100000000000000E842
:101B4000FFFFFF00000000000000000000FAFFFFA0
:101B50003F0000000000000000FFFFFFFFFF7F00CC
:101B600000000000000000FAFFFF1F00000000005E
:101B70000000000000F0FFFFFF0000000000000078
:101B800000FEFFFFFFFFFF0000000000000000FE5E
:101B9000FFFF1F00000000000000000000E8FFFF42
:101BA000FF0300000000000000FCFFFFFFFF3F00FC
:101BB000000000000000C0FFFFFF07000000000061
:101BC0000000000000C0FFFFFF0F00000000000049
:101BD00000F8FFFFFFFF3F00000000000000D0FF03
:101BE000FFFF0F0000000000000000000040FFFFAA
:101BF000FF3700000000000000F4FFFFFFFF1F00A0
:101C0000000000000000F4FFFFFF010000000000E2
:101C1000000000000000FFFFFFFF000000000000C8
:101C200000F0FFFFFFFF1F00000000000000FDFFAD
:101C3000FF7F010000000000000000000000FEFF28
:101C4000FF7F03000000000000F0FFFFFFFF070020
:101C5000000000000040FFFFFF7F000000000000C8
:101C6000000000000000F8FFFFFF0F000000000070
:101C700000C0FFFFFFFF0F000000000000E8FFFFB3
:101C8000FF5F000000000000000000000000F0FF07
:101C9000FFFF3F000000000000E0FFFFFFFF030028
:101CA0000000000000FAFFFFFF0F0000000000002E
:101CB000000000000000C0FFFFFFFF030000000065
:101CC0000080FFFFFFFF03000000000080FEFFFF19
:101CD000FF0B000000000000000000000000A0FF5B
:101CE000FFFFFF0D000000000080FFFFFFFF01006D
:101CF00000000000E8FFFFFFFF05000000000000FB
:101D000000000000000000FFFFFFFFBF0000000018
:101D10000000FFFFFFFF010000000000FAFFFFFFCF
:101D2000FF0100000000000000000000000000FCB7
:101D3000FFFFFFFF0B0000000000FFFFFF7F000020
:101D4000000000D0FFFFFFFF3F0000000000000088
:101D500000000000000000F8FFFFFFFFBF000000D0
:101D60000000FEFFFFFF0000000000FAFFFFFFFF82
:101D70003F0000000000000000000000000000D054
:101D8000FFFFFFFFFF1700000000FCFFFF3F000008
:101D90000000F4FFFFFFFFFF07000000000000004D
:101DA00000000000000000A0FFFFFFFFFFFF2A006F
:101DB0000000FCFFFF7F000000A8EDFFFFFFFFFF1A
:101DC000050000000000000000000000000000808E
:101DD000FEFFFFFFFFFFEF2A0991FAFFFFBF089107
:101DE000D4FBFFFFFFFFFFFF020000000000000028
:101DF0000000000000000000FCFFFFFFFFFFFFFFEE
:101E00007FB7FFFFFFFF7BFFBFFFFFFFFFFFFF7FEE
:101E100000000000000000000000000000000000C2
:101E2000F2FFFFFFFFFFFFFFFFFFFFFFFFFFFFFFCF
:101E3000FFFFFFFFFFFFFF0F00000000000000009A
:101E40000000000000000000C0FFFFFFFFFFFFFFD9
:101E5000FFFFFFFFFFFFFFFFFFFFFFFFFFFFFF177A
:101E60000000000000000000000000000000000072
:101E7000A0FFFFFFFFFFFFFFFFFFFFFFFFFFFFFFD1
:101E8000FFFFFFFFFFFFFF00000000000000000059
:101E9000000000000000000000FCFFFFFFFFFFFF4C
:101EA000FFFFFFFFFFFFFFFFFFFFFFFFFFFF7F01C0
:101EB0000000000000000000000000000000000022
:101EC00000F0FFFFFFFFFFFFFFFFFFFFFFFFFFFF30
:101ED000FFFFFFFFFFFF0F000000000000000000F9
:101EE000000000000000000000A0FFFFFFFFFFFF58
:101EF000FFFFFFFFFFFFFFFFFFFFFFFFFFFF0B00E5
:101F000000000000000000000000000000000000D1
:101F10000080FEFFFFFFFFFFFFFFFFFFFFFFFFFF50
:101F2000FFFFFFFFFF7F0000000000000000000037
:101F300000000000000000000000F4FFFFFFFFFFB2
:101F4000FFFFFFFFFFFFFFFFFFFFFFFFFF5F00003F
:101F50000000000000000000000000000000000081
:101F60000000C0FFFFFFFFFFFFFFFFFFFFFFFFFFBE
:101F7000FFFFFFFFFF010000000000000000000065
:101F80000000000000000000000000FCFFFFFFFF59
:101F9000FFFFFFFFFFFFFFFFFFFFFFFFBF0200008C
:101FA0000000000000000000000000000000000031
:101FB000000000D2FFFFFFFFFFFFFFFFFFFFFFFF5B
:101FC000FFFFFFFF0B00000000000000000000000A
:101FD000000000000000000000000000FDFFFFFF07
:101FE000FFFFFFFFFFFFFFFFFFFFFFBF020000003B
:101FF00000000000000000000000000000000000E1
:1020000000000000D0FFFFFFFFFFFFFFFFFFFFFF0B
:10201000FFFFFF0B000000000000000000000000B8
:1020200000000000000000000000000000FAFFFFB8
:10203000FFFFFFFFFFFFFFFFFFFF5F20000000002B
:102040000000000000000000000000000000000090
:10205000000000000000FDFFFFFFFFFFFFFFFFFF8C
:10206000FF5F000000000000000000000000000012
:10207000000000000000000000000000000000AAB6
:102080006DDBB62A526DDBB6554101000000000041
:102090000000000000000000000000000000000040
:1020A00000000000000040409024080000902449F7
:1020B000040000000000000000000000000000001C
:1020C0000000000000000000000000000000000010
:1020D00000002000000000000000000000000000E0
:1020E00000000000000000000000000000000000F0
:1020F00000000000000000000000000000000000E0
:1021000000000000000000000000000000000000CF
:1021100000000000000000000000000000000000BF
:1021200000000000000000000000000000000000AF
:10213000000000000000000000000000000000009F
:10214000000000000000000000000000000000008F
:10215000000000000000000000000000000000007F
:10216000000000000000000000000000000000006F
:10217000000000000000000000000000000000005F
:10218000000000000000000000000000000000004F
:10219000000000000000000000000000000000003F
:1021A000000000000000000000000000000000002F
:1021B000000000000000000000000000000000001F
:1021C000000000000000000000000000000000000F
:1021D00000000000000000000000000000000000FF
:1021E00000000000000000000000000000000000EF
:1021F00000000000000000000000000000000000DF
:1022000000000000000000000000000000000000CE
:1022100000000000000000000000000000000000BE
:10222000000000000000000000000A0B02090C0D75
:102230000E08070304010000000000000000000079
:10224000000000000000000000000000000000008E
:10225000000000001211100000000000000000004B
:10226000000000000000000000000000000000006E
:102270000000003E5B4F5B3E3E6B4F6B3E1C3E7C66
:102280003E1C183C7E3C181C577D571C1C5E7F5E14
:102290001C00183C1800FFE7C3E7FF0018241800D3
:1022A000FFE7DBE7FF30483A060E2629792926406A
:1022B0007F050507407F05253F5A3CE73C5A7F3E96
:1022C0001C1C08081C1C3E7F14227F22145F5F0028
:1022D0005F5F06097F017F006689956A60606060C4
:1022E0006094A2FFA29408047E040810207E2010AF
:1022F00008082A1C08081C2A08081E101010100CB8
:102300001E0C1E0C30383E3830060E3E0E06000005
:1023100000000000005F00000007000700147F14A9
:102320007F14242A7F2A1223130864623649562018
:10233000500008070300001C2241000041221C003D
:102340002A1C7F1C2A08083E0808008070300008FC
:1023500008080808000060600020100804023E51D0
:1023600049453E00427F4000724949494621414962
:102370004D331814127F1027454545393C4A4949C9
:102380003141211109073649494936464949291E33
:102390000000140000004034000000081422411422
:1023A00014141414004122140802015909063E4174
:1023B0005D594E7C1211127C7F494949363E41419C
:1023C00041227F4141413E7F494949417F090909F5
:1023D000013E414151737F0808087F00417F410061
:1023E0002040413F017F081422417F404040407F10
:1023F000021C027F7F0408107F3E4141413E7F095D
:102400000909063E4151215E7F091929462649499D
:10241000493203017F01033F4040403F1F204020DD
:102420001F3F4038403F63140814630304780403DB
:102430006159494D43007F41414102040810200089
:102440004141417F040201020440404040400003FA
:1024500007080020545478407F28444438384444C6
:102460004428384444287F385454541800087E09BE
:102470000218A4A49C787F0804047800447D4000DE
:102480002040403D007F1028440000417F40007CF8
:10249000047804787C080404783844444438FC18F0
:1024A00024241818242418FC7C08040408485454D4
:1024B000542404043F44243C4040207C1C20402001
:1024C0001C3C4030403C44281028444C9090907C68
:1024D0004464544C4400083641000000770000007A
:1024E0004136080002010204023C2623263C1EA1BC
:1024F000A161123A4040207A38545455592155551B
:1025000079412254547842215554784020545579C9
:10251000400C1E527212395555555939545454595C
:1025200039555454580000457C410002457D420015
:1025300001457C407D1211127DF0282528F07C5445
:102540005545002054547C547C0A097F493249493E
:1025500049323A4444443A324A4848303A414121A7
:102560007A3A42402078009DA0A07D3D4242423D03
:102570003D4040403D3C24FF2424487E4943662B97
:102580002FFC2F2BFF0929F620C0887E0903205439
:102590005479410000447D413048484A3238404037
:1025A000227A007A0A0A727D0D19317D2629292F97
:1025B00028262929292630484D40203808080808AF
:1025C00008080808382F10C8ACBA2F102834FA00B1
:1025D000007B000008142A142222142A1408550033
:1025E000550055AA55AA55AAFF55FF55FF000000F2
:1025F000FF00101010FF00141414FF001010FF0053
:10260000FF1010F010F0141414FC001414F700FF65
:102610000000FF00FF1414F404FC141417101F1022
:10262000101F101F1414141F00101010F0000000D1
:10263000001F101010101F10101010F010000000DC
:10264000FF101010101010101010FF10000000FFED
:10265000140000FF00FF00001F10170000FC04F42E
:1026600014141710171414F404F40000FF00F714E6
:10267000141414141414F700F7141414171410106D
:102680001F101F141414F4141010F010F000001F89
:10269000101F0000001F14000000FC140000F010C8
:1026A000F01010FF10FF141414FF141010101F006E
:1026B000000000F010FFFFFFFFFFF0F0F0F0F0FF70
:1026C000FFFF0000000000FFFF0F0F0F0F0F384447
:1026D000443844FC4A4A4A347E02020606027E021C
:1026E0007E0263554941633844443C04407E201EC9
:1026F0002006027E020299A5E7A5991C2A492A1CF8
:102700004C7201724C304A4D4D303048784830BCE4
:10271000625A463D3E494949007E0101017E2A2A0E
:102720002A2A2A44445F444440514A444040444A8F
:1027300051400000FF0103E080FF000008086B6BC0
:10274000083612362436060F090F06000018180046
:1027500000001010003040FF0101001F01011E00A9
:10276000191D1712003C3C3C3C000000000000001A
:102770002100240027002A002D0030003300010131
:102780000000040107010A010102102020080810BE
:1027900020401020408002010201080402010102D1
:1027A00004081020408080402010080402018004AA
:1027B0000201804020100804020108040201010205
:1027C000040810204080010204081020408000000E
:1027D0002200250028002B002E00310034000201C9
:1027E0000000050108010B0105050505070508089E
:1027F0000808020202020A0A08080404040401018B
:10280000010101010101030303030303030304079F
:1028100007070C0C0C0C0C0C0C0C02020202060636
:102820000606060606060B0B0B0B0B0B0B0B1430E8
:102830004D2B11241FBECFEFD1E2DEBFCDBF00E094
:102840000CBF2DE0AAE0BDE001C01D92A63EB2077C
:10285000E1F71DE0A0E0B2E0ECE1F7E600E00BBF3D
:1028600002C007900D92AA30B107D9F714E1C8E170
:10287000D4E100E006C021970109802FFE010E94EB
:102880002231C731D10780E00807A9F70E94512BF8
:102890000C947D330C9400000895FC016370658BEB
:1028A0008481958126813781613039F0633029F048
:1028B0009187808733872287089531872087938780
:1028C000828708956F927F928F929F92AF92BF926C
:1028D000CF92DF92EF92FF920F931F93CF93DF93EC
:1028E000EC014B015A0169013801E881F981028448
:1028F000F385E02D1995E881F9810288F389E02DAF
:1029000087019601A501B401CE011995A501460DD7
:10291000571D41505109E881F9810288F389E02D62
:102920009601B401CE011995E881F9810088F189F9
:10293000E02D9301A501B401CE011995C80CD91C55
:10294000B60161507109E881F9810088F189E02DB3
:102950009301A501CE011995E881F9810688F789CF
:10296000E02DCE01DF91CF911F910F91FF90EF905D
:10297000DF90CF90BF90AF909F908F907F906F909F
:1029800019948F929F92AF92BF92CF92DF92EF9263
:10299000FF920F931F93CF93DF934C016B015A016A
:1029A000E901DC01ED91FC916217730781F40417D2
:1029B000150724F48B2D5801042F182F0A191B0911
:1029C00098012F5F3F4F048CF58DE02D12C040170A
:1029D000510709F52617370724F48D2D6901C62FF5
:1029E000D82F9E012C193D092F5F3F4F068CF78D84
:1029F000E02D8701A501B601C4011995DF91CF91A2
:102A00001F910F91FF90EF90DF90CF90BF90AF900C
:102A10009F908F9008950284F385E02D1995D4013D
:102A2000ED91FC910488F589E02D9E01A501B60188
:102A3000C4011995D401ED91FC910688F789E02D28
:102A4000C401DF91CF911F910F91FF90EF90DF9024
:102A5000CF90BF90AF909F908F901994EF92FF927C
:102A60000F931F93DC011A960D911C911B971896DA
:102A70002D913C911997ED91FC9100A0F1A1E02DD1
:102A80007B0140E050E060E070E019951F910F91EC
:102A9000FF90EF9008954F925F926F927F928F9286
:102AA0009F92AF92BF92CF92DF92EF92FF920F93DD
:102AB0001F93CF93DF936C012B015A013901480119
:102AC000DC01ED91FC910284F385E02D1995E20182
:102AD000640C751CD601ED91FC91C615D7055CF40C
:102AE0000088F189E02D87019401A501BE01C6018E
:102AF00019952196EFCF0688F789E02DC601DF9161
:102B0000CF911F910F91FF90EF90DF90CF90BF90EA
:102B1000AF909F908F907F906F905F904F9019949F
:102B20008F929F92AF92BF92CF92DF92EF92FF92DD
:102B30000F931F93CF93DF93EC015B014A0169016F
:102B4000E881F9810284F385E02D199595012C0D1A
:102B50003D1D21503109E881F9810488F589E02D76
:102B600078018401A401B501CE011995E881F981AC
:102B70000688F789E02DCE01DF91CF911F910F914B
:102B8000FF90EF90DF90CF90BF90AF909F908F908D
:102B900019948F929F92AF92BF92CF92DF92EF9251
:102BA000FF920F931F93CF93DF93EC015B014A01D8
:102BB00069017801E881F9810284F385E02D199596
:102BC000C80CD91C860101501109E881F9810488DB
:102BD000F589E02D9501A401B501CE011995E88193
:102BE000F9810688F789E02DCE01DF91CF911F9101
:102BF0000F91FF90EF90DF90CF90BF90AF909F909C
:102C00008F9019940895EF92FF920F931F93DC0118
:102C1000ED91FC9100A0F1A1E02D19951F910F916C
:102C2000FF90EF9008950F931F93DC01ED91FC91BD
:102C3000068CF78DE02D19951F910F9108950F9334
:102C40001F93DC01ED91FC91048CF58DE02D19951D
:102C50001F910F910895DC01ED91FC910084F185A5
:102C6000E02D19942F923F924F925F926F927F9234
:102C70008F929F92AF92BF92CF92DF92EF92FF928C
:102C80000F931F93CF93DF9300D000D0CDB7DEB763
:102C90002C017E836D836A015901C801FC82EB829D
:102CA0004801841A950A97FE03C091948194910873
:102CB00035012D813E81621A730A77FE03C071943B
:102CC00061947108681479045CF43A2D2B2D5C0131
:102CD000832F922F3D812E81DE82CD82C32ED22E74
:102CE000AD81BE81AA16BB065CF43C2D2D2D6C0176
:102CF000832F922F3D812E81BE82AD82A32EB22ED4
:102D000085012D813E81021B130B1C012C183D08EF
:102D100037FE03C0319421943108780117FF03C0B6
:102D20003FEFE31AF30AF594E794C816D9062CF09E
:102D30008FEF9FEF9A83898304C0A1E0B0E0BA834C
:102D4000A9832D813E81A216B30624F1D201ED9113
:102D5000FC910484F585E02D2B813C816814790475
:102D600024F44D815E81B60103C0A6016D817E8190
:102D7000C2011995E218F308F7FE06C029813A81CD
:102D8000C20ED31EE00EF11E8D819E8101969E83A0
:102D90008D83D7CF26960FB6F894DEBF0FBECDBF7A
:102DA000DF91CF911F910F91FF90EF90DF90CF9027
:102DB000BF90AF909F908F907F906F905F904F905B
:102DC0003F902F900895089580E090E00895AF928D
:102DD000BF92CF92EF92FF920F931F93CF93DF9307
:102DE000EC01262F888D998D009709F040C06A303C
:102DF00059F41D861C862C898E859F8538E0239F7B
:102E0000800D911D112441C06D3009F4AAC08E8936
:102E10008823C1F03C898C859D8546E0349F800DD8
:102E2000911D112448855985481759075CF41D8662
:102E30001C868E859F8548E0349F800D911D11244E
:102E40009F878E87EA88FB88088919894E855F8568
:102E50006C857D85CC88CE010E94A2242C898C852E
:102E60009D8536E0239F800D911D112442C06A305C
:102E700079F41D861C862C89FC013696E4918E859A
:102E80009F852E9F800D911D11249F878E8769C07D
:102E90006D3009F466C0FC0134963491631708F470
:102EA00060C03196E491E61708F45BC0FC013296ED
:102EB00065917491422F50E0431B510937E0349FD4
:102EC0005001359FB00C1124A60EB71EF5013296A5
:102ED00034913196E491332311F0E1110DC0F501E5
:102EE0003496E4912C898C859D85E29F800D911DFF
:102EF00011249D878C8735C0F501359644915E89F4
:102F0000552311F16C89E32FF0E0E40FF11D47FD2B
:102F1000FA956E9FD0016F9FB00D11244C855D8591
:102F20004A0F5B1FE885F985E417F5076CF41D86E9
:102F30001C86FC013696E4918E859F856E9F800DE0
:102F4000911D11249F878E87EA88FB88088919893B
:102F50004E855F856C857D85CC88CE010E94A2243C
:102F6000BECF81E090E0DF91CF911F910F91FF9054
:102F7000EF90CF90BF90AF900895FC01A38DB48DDA
:102F80009C9187A189238C93808591859C012150F8
:102F900031098150A58DB68D2C9190A592239C93DB
:102FA00094E092B9A78DB0A12C9191A592239C9306
:102FB000A78DB0A12C9195A1922B9C93A58DB68D38
:102FC0002C9194A1922B9C9332B9A78DB0A12C91F6
:102FD00091A592239C93A78DB0A12C9195A1922BA2
:102FE0009C93A58DB68D2C9190A592239C9395E0F2
:102FF00092B9A78DB0A12C9191A592239C93A78DF6
:10300000B0A12C9195A1922B9C93A58DB68D2C915E
:1030100094A1922B9C9382B9A78DB0A19C9181A57C
:1030200089238C93A78DB0A19C9185A1892B8C932A
:10303000828593859C01215031098150A58DB68DE3
:103040002C9190A592239C9398E092B9A78DB0A162
:103050002C9191A592239C93A78DB0A12C9195A121
:10306000922B9C93A58DB68D2C9194A1922B9C9321
:1030700032B9A78DB0A12C9191A592239C93A78DD5
:10308000B0A12C9195A1922B9C93A58DB68D2C91DE
:1030900090A592239C9399E092B9A78DB0A12C9111
:1030A00091A592239C93A78DB0A12C9195A1922BD1
:1030B0009C93A58DB68D2C9194A1922B9C9382B953
:1030C000A78DB0A19C9181A589238C93A78DB0A1D8
:1030D0009C9185A1892B8C93A38DB48D9C9183A108
:1030E000892B8C930895EF92FF920F931F93CF93A8
:1030F000DF93EC01CB017A01EB8DFC8D50814FA168
:10310000452340834A8D4111B6C14D89423089F033
:10311000433021F1413091F54FEE50E0DA01A01B30
:10312000B10B4E195F09FA0189019A017B01CD01AA
:1031300027C06FEE70E0AB01421B530B9B01281BB5
:10314000390B8FE391E0DC01A01BB10B8C010E1950
:103150001F09B801F9017D01CA0112C04FE351E016
:10316000DA01A21BB30B9A01261B370BC901B90167
:10317000F70198018C01C7017D0102C0B701FC0174
:10318000AD8DBE8D5C9148A545234C9312B8AF8D93
:10319000B8A15C9149A545234C93AF8DB8A15C9132
:1031A0004DA1452B4C9340E542B9AF8DB8A15C9140
:1031B00049A545234C93AF8DB8A15C914DA1452BFA
:1031C0004C93AD8DBE8D5C914CA1452B4C9392B927
:1031D000AF8DB8A14C9199A594239C93AF8DB8A1C4
:1031E0004C919DA1942B9C9382B9AF8DB8A19C91D9
:1031F00089A589238C93AF8DB8A19C918DA1892B32
:103200008C93AD8DBE8D9C9188A589238C9312B82B
:10321000AF8DB8A19C9189A589238C93AF8DB8A15E
:103220009C918DA1892B8C9381E582B9AF8DB8A13A
:103230009C9189A589238C93AF8DB8A19C918DA178
:10324000892B8C93AD8DBE8D9C918CA1892B8C93F9
:1032500032B9AF8DB8A19C9189A589238C93AF8D8C
:10326000B8A19C918DA1892B8C9322B9AF8DB8A167
:103270009C9189A589238C93AF8DB8A19C918DA138
:10328000892B8C93AD8DBE8D9C9188A589238C93C1
:1032900012B8AF8DB8A19C9189A589238C93AF8D6D
:1032A000B8A19C918DA1892B8C9382E582B9AF8DB9
:1032B000B8A19C9189A589238C93AF8DB8A19C91CD
:1032C0008DA1892B8C93AD8DBE8D9C918CA1892B6A
:1032D0008C93F2B8AF8DB8A19C9189A589238C936A
:1032E000AF8DB8A19C918DA1892B8C93E2B8AF8D45
:1032F000B8A19C9189A589238C93AF8DB8A19C918D
:103300008DA1892B8C93AD8DBE8D9C9188A5892331
:103310008C9312B8AF8DB8A19C9189A589238C9309
:10332000AF8DB8A19C918DA1892B8C9383E582B937
:10333000AF8DB8A19C9189A589238C93AF8DB8A13D
:103340009C918DA1892B8C93AD8DBE8D9C918CA170
:10335000892B8C9312B9AF8DB8A19C9189A5892333
:103360008C93AF8DB8A19C918DA1892B8C9302B9C0
:10337000AF8DB8A19C9189A589238C93AF8DB8A1FD
:103380009C918DA1892B8C93AD8DBE8D9C9188A530
:1033900089238C9312B8AF8DB8A19C9189A58923FC
:1033A0008C93AF8DB8A19C918DA1892B8C9380E2D9
:1033B00082B9AF8DB8A19C9189A589238C93AF8DDB
:1033C000B8A19C918DA1892B8C93AD8DBE8D9C91C4
:1033D0008CA1892B8C93F2B9AF8DB8A19C9189A552
:1033E00089238C93AF8DB8A19C918DA1892B8C934F
:1033F000E2B9EF8DF8A1908189A589238083EF8DB3
:10340000F8A190818DA1892B8083ED8DFE8D908117
:1034100088A58923808312B8EF8DF8A1908189A5B2
:1034200089238083EF8DF8A190818DA1892B8083E2
:1034300081E282B9EF8DF8A1908189A589238083EB
:10344000EF8DF8A190818DA1892B8083ED8DFE8D6C
:1034500090818CA1892B808372B9EF8DF8A1908126
:1034600089A589238083EF8DF8A190818DA1892B77
:10347000808362B92FC1413009F039C1ED8DFE8DD5
:10348000508148A54523408342E042B9EF8DF8A121
:10349000508149A545234083EF8DF8A150814DA16E
:1034A000452B4083ED8DFE8D50814CA1452B4083F3
:1034B00092B9EF8DF8A1408199A594239083EF8D67
:1034C000F8A140819DA1942B9083ED8DFE8D4081CC
:1034D00098A59423908393E092B9EF8DF8A1408151
:1034E00099A594239083EF8DF8A140819DA1942B01
:1034F0009083ED8DFE8D40819CA1942B908382B9A9
:10350000EF8DF8A1908189A589238083EF8DF8A1A3
:1035100090818DA1892B8083ED8DFE8D908188A572
:103520008923808386E082B9EF8DF8A1908189A5F7
:1035300089238083EF8DF8A190818DA1892B8083D1
:10354000ED8DFE8D90818CA1892B8083F2B8EF8D5B
:10355000F8A1908189A589238083EF8DF8A19081BE
:103560008DA1892B8083ED8DFE8D908188A5892387
:10357000808387E082B9EF8DF8A1908189A58923A6
:103580008083EF8DF8A190818DA1892B8083ED8DB3
:10359000FE8D90818CA1892B8083E2B8EF8DF8A1FC
:1035A000908189A589238083EF8DF8A190818DA1D9
:1035B000892B8083ED8DFE8D908188A58923808362
:1035C00084E082B9EF8DF8A1908189A58923808359
:1035D000EF8DF8A190818DA1892B8083ED8DFE8DDB
:1035E00090818CA1892B808332B9EF8DF8A19081D5
:1035F00089A589238083EF8DF8A190818DA1892BE6
:103600008083ED8DFE8D908188A58923808385E060
:1036100082B9EF8DF8A1908189A589238083EF8DF0
:10362000F8A190818DA1892B8083ED8DFE8D9081F5
:103630008CA1892B808322B9EF8DF8A1908189A577
:1036400089238083EF8DF8A190818DA1892B8083C0
:10365000ED8DFE8D908188A58923808388E082B9D5
:10366000EF8DF8A1908189A589238083EF8DF8A142
:1036700090818DA1892B8083ED8DFE8D90818CA111
:10368000892B808312B9EF8DF8A1908189A58923B8
:103690008083EF8DF8A190818DA1892B8083ED8DA2
:1036A000FE8D908188A58923808389E082B9EF8D82
:1036B000F8A1908189A589238083EF8DF8A190815D
:1036C0008DA1892B8083ED8DFE8D90818CA1892B1E
:1036D000808302B9EF8DF8A1908189A58923808329
:1036E000EF8DF8A190818DA1892B80832FC042504E
:1036F000423060F5092E000CAA0BBB0BDC019927A8
:103700008827A901330F660B770B9A01AB01282B91
:10371000392B4A2B5B2B6AE2CE010E942724C7017A
:10372000FF0CAA0BBB0BBC0155274427012E000C34
:10373000220B330BD901C801842B952BA62BB72B59
:103740009C01AD016BE2CE010E942724EB8DFC8D24
:1037500090818BA1892B8083DF91CF911F910F9155
:10376000FF90EF900895EF92FF920F931F93CF93E6
:10377000DF93EC017B018A8D81119DC0ED89E150C1
:10378000E33060F4F0E0DF01A45FBD4F8C91EE0FF9
:10379000FF1FEA5FFD4F2081318104C020E030E04F
:1037A00080E090E0EB8DFC8D40819FA1942390837D
:1037B000ED8DFE8D408198A59423908312B8EF8DF6
:1037C000F8A1408199A594239083EF8DF8A14081C1
:1037D0009DA1942B908390E292B9EF8DF8A1408146
:1037E00099A594239083EF8DF8A140819DA1942BFE
:1037F0009083ED8DFE8D40819CA1942B908312B817
:10380000EF8DF8A1408199A594239083EF8DF8A1C5
:1038100040819DA1942B908382B9EF8DF8A1908176
:1038200089A589238083EF8DF8A190818DA1892BB3
:103830008083ED8DFE8D908188A58923808312B8C9
:10384000EF8DF8A1908189A589238083EF8DF8A160
:1038500090818DA1892B808381E282B9EF8DF8A1BF
:10386000908189A589238083EF8DF8A190818DA116
:10387000892B8083ED8DFE8D90818CA1892B808397
:1038800032B9EF8DF8A1908189A589238083EF8DCE
:10389000F8A190818DA1892B808322B9EF8DF8A1A9
:1038A000908189A589238083EF8DF8A190818DA1D6
:1038B000892B808311C08150833070F40A851B8569
:1038C00001501109288539852150310940E050E027
:1038D00060E070E0CE0107DC20E03CE241E050E037
:1038E000B701CE01DF91CF911F910F91FF90EF9023
:1038F0000C94B4298F929F92AF92BF92CF92DF9295
:10390000EF92FF920F931F93CF93DF93EC01470148
:10391000121613060CF068C0101611060CF064C0E5
:10392000A885B9856A177B070CF05EC0CA84DB8462
:103930004C155D050CF058C07901E60EF71EC70165
:10394000019797FD51C05801A40EB51EF50131979E
:10395000F7FD4AC077FF46C060E070E057FD02C047
:10396000580102C040E050E08A179B072CF0CD01BF
:1039700001977D01E61AF70AEC15FD052CF0F6011A
:1039800031975601A41AB50A8F019C01CE01ABDB19
:103990009701D5010E942A319B01AC01B401CE01EF
:1039A0000E94B4298A8D81110FC00A851B850150A0
:1039B0001109288539852150310940E050E060E047
:1039C00070E0CE0190DB10C0CE01DF91CF911F914E
:1039D0000F91FF90EF90DF90CF90BF90AF909F90AE
:1039E0008F90CBCA7901BACFDF91CF911F910F9100
:1039F000FF90EF90DF90CF90BF90AF909F908F900F
:103A00000895CF92DF92EF92FF920F931F93CF937F
:103A1000DF93EC016801121613060CF04CC077FD21
:103A20004AC088859985681779070CF044C08A8553
:103A30009B85481759070CF03EC07901E40EF51E2E
:103A400087010150110917FD36C057FF32C040E011
:103A500050E00817190734F08C01015011097C015E
:103A6000E41AF50A9B01CE013EDB9701FF0C440BE3
:103A7000550BB601CE010E94B4298A8D81110FC069
:103A80000A851B8501501109288539852150310986
:103A900040E050E060E070E0CE0125DB0CC0CE01DC
:103AA000DF91CF911F910F91FF90EF90DF90CF901A
:103AB00064CA7901CECFDF91CF911F910F91FF9012
:103AC000EF90DF90CF900895CF92DF92EF92FF9228
:103AD0000F931F93CF93DF93EC0168011216130627
:103AE0000CF04BC057FD49C08A859B854817590784
:103AF0000CF043C0E885F9856E177F070CF03DC0D8
:103B00007901E60EF71EC701019797FD36C077FFD2
:103B100032C060E070E08E179F072CF0CF01019754
:103B20007F01E61AF70A8A019C01CE01DCDA9701CF
:103B3000FF0C440B550BB601CE010E94B4298A8DAF
:103B400081110FC00A851B8501501109288539850F
:103B50002150310940E050E060E070E0CE01C3DA6E
:103B60000CC0CE01DF91CF911F910F91FF90EF908C
:103B7000DF90CF9002CA7901CECFDF91CF911F9114
:103B80000F91FF90EF90DF90CF9008950E94373310
:103B90000F931F93CF93DF93EC0188819981009756
:103BA00029F02A813B812617370788F48B016F5F44
:103BB0007F4F0E945732009761F0998388831B835F
:103BC0000A832C813D81232B11F4FC01108281E0BA
:103BD00001C080E0DF91CF911F910F9108953FB711
:103BE000F89480910F0D9091100DA091110DB0914E
:103BF000120D26B5A89B05C02F3F19F00196A11DF7
:103C0000B11D3FBFBA2FA92F982F8827820F911D72
:103C1000A11DB11DBC01CD0142E0660F771F881FB9
:103C2000991F4A95D1F708951F920F920FB60F92E0
:103C300011242F933F938F939F93AF93BF938091C2
:103C40000B0D90910C0DA0910D0DB0910E0D3091BA
:103C50000A0D23E0230F2D3720F40196A11DB11D7D
:103C600005C026E8230F0296A11DB11D20930A0D61
:103C700080930B0D90930C0DA0930D0DB0930E0D32
:103C800080910F0D9091100DA091110DB091120D1A
:103C90000196A11DB11D80930F0D9093100DA0935F
:103CA000110DB093120DBF91AF919F918F913F91E4
:103CB0002F910F900FBE0F901F901895EF92FF92CB
:103CC0000F931F93CF93DF936115710511F480E07B
:103CD0001BC041155105B9F07B01EC018C819D8120
:103CE0008A01080F191FB801CE0152DF882379F32A
:103CF000288139818C819D81B701820F931F0E9499
:103D00004D331D830C8381E0DF91CF911F910F9183
:103D1000FF90EF900895FB0144815581608171818E
:103D2000CDCFCF93DF93EC0188819981009711F07B
:103D30000E94CE31198218821D821C821B821A8237
:103D4000DF91CF910895EF92FF920F931F93CF933E
:103D5000DF93EC017B018A01BA011ADF811103C0F4
:103D6000CE01DFDF07C01D830C83B70188819981F5
:103D70000E944D33CE01DF91CF911F910F91FF90A3
:103D8000EF900895FC01808191810C94CE31FB016C
:103D9000DC0111961C921E9213961C921E92129791
:103DA00015961C921E9214978617970741F0608112
:103DB00071816115710519F044815581C4CF089551
:103DC000FC01118210821382128215821482611505
:103DD000710549F0FB0101900020E9F73197AF012F
:103DE000461B570BB0CF0895BF92CF92DF92EF9250
:103DF000FF920F931F93CF93DF937C016B01EA0136
:103E000089012417350720F48D2FE901042F182F7D
:103E100068E07DE0C701D4DFD60114968D919C91B6
:103E20001597C817D90730F58017910708F48C014A
:103E3000D601ED91FC911197E00FF11FB080108237
:103E40006D917C916C0F7D1F6115710559F0FB011F
:103E500001900020E9F73197AF01461B570BC701CE
:103E600072DF02C0C7015DDFD601ED91FC91E00F6A
:103E7000F11FB082C701DF91CF911F910F91FF9089
:103E8000EF90DF90CF90BF900895CF92DF92EF92A6
:103E9000FF920F931F93CF93DF936C017A018B01F5
:103EA000C0E0D0E0CE15DF0581F0D8016D918D0125
:103EB000D601ED91FC910190F081E02DC60119959C
:103EC000892B11F02196EECF7E01C701DF91CF91B2
:103ED0001F910F91FF90EF90DF90CF900895FC011C
:103EE000538D448D252F30E0842F90E0821B930B5F
:103EF000541710F0CF96089501970895FC01918D05
:103F0000828D981761F0828DDF01A80FB11D5D963B
:103F10008C91928D9F5F9F73928F90E008958FEFA9
:103F20009FEF0895FC01918D828D981731F0828D5D
:103F3000E80FF11D858D90E008958FEF9FEF0895B4
:103F4000FC01918D228D892F90E0805C9F4F821B18
:103F500091098F739927089583E19DE0F1DF21E0B6
:103F6000892B09F420E0822F0895FC01848DDF0164
:103F7000A80FB11DA35ABF4F2C91848D90E00196DC
:103F80008F739927848FA689B7892C93A089B189CB
:103F90008C91837080648C93938D848D981306C06C
:103FA0000288F389E02D80818F7D80830895EF92D0
:103FB000FF920F931F93CF93DF93EC0181E0888FE3
:103FC0009B8D8C8D981305C0E889F989808185FDCA
:103FD00025C0F62E0B8D10E00F5F1F4F0F731127BA
:103FE000E02E8C8DE8120BC00FB607FCFACFE889E3
:103FF000F989808185FFF5CFCE01B7DFF2CF8B8DB8
:10400000FE01E80FF11DE35AFF4FF0829FB7F894CD
:104010000B8FEA89FB89808180620AC09FB7F89480
:10402000EE89FF896083E889F989808183708064E3
:1040300080839FBF81E090E0DF91CF911F910F912E
:10404000FF90EF900895CF93DF93EC01888D882344
:10405000C1F0EA89FB89808185FD05C0A889B989FD
:104060008C9186FD0EC00FB607FCF5CF808185FFD1
:10407000F2CFA889B9898C9185FFEDCFCE0175DF8C
:10408000E8CFDF91CF91089580E090E0892B19F07F
:1040900063DF811125C080E090E0892B41F080E052
:1040A00090E0892B21F00E94000081111CC080E06B
:1040B00090E0892B41F080E090E0892B21F00E9474
:1040C0000000811113C080E090E0892BA1F080E016
:1040D00090E0892B81F00E94000081110AC00895B0
:1040E0000E940000D8CF0E940000E1CF0E94000093
:1040F000EACF0C9400000895EF92FF920F931F9364
:10410000CF93DF93EC01F22EE32E77FDF4C157FD40
:10411000F2C188859985681779070CF0ECC18A850A
:104120009B85481759070CF0E6C1EB8DFC8D9081FB
:104130008FA1892380838A8D8111B6C08D898230B9
:1041400059F08330B1F08130D1F48FEE90E0841BD0
:10415000950BAB01BC0113C08FEE90E09C01261BB8
:10416000370BB9018FE391E09C01241B350BA901AA
:1041700006C08FE391E0861B970BBA01AC01ED8D71
:10418000FE8D908188A58923808312B8EF8DF8A1D8
:10419000908189A589238083EF8DF8A190818DA1DD
:1041A000892B808380E282B9EF8DF8A1908189A567
:1041B00089238083EF8DF8A190818DA1892B808345
:1041C000ED8DFE8D90818CA1892B808372B9EF8D4E
:1041D000F8A1908189A589238083EF8DF8A1908132
:1041E0008DA1892B808362B9EF8DF8A1908189A57B
:1041F00089238083EF8DF8A190818DA1892B808305
:10420000ED8DFE8D908188A58923808312B8EF8D76
:10421000F8A1908189A589238083EF8DF8A19081F1
:104220008DA1892B808381E282B9EF8DF8A19081E5
:1042300089A589238083EF8DF8A190818DA1892B99
:104240008083ED8DFE8D90818CA1892B808352B966
:10425000EF8DF8A1908189A589238083EF8DF8A146
:1042600090818DA1892B808342B9EF8DF8A1908137
:1042700089A589238083EF8DF8A190818DA1892B59
:104280008083ED8DFE8D908188A58923808312B86F
:10429000EF8DF8A1908189A589238083EF8DF8A106
:1042A00090818DA1892BD5C0813009F0D5C0ED89D1
:1042B000E150E33028F4F0E0E15FFD4F908101C070
:1042C00090E0ED8DFE8D208188A58223808386E19C
:1042D00082B9EF8DF8A1208189A582238083EF8D9B
:1042E000F8A120818DA1822B8083ED8DFE8D208110
:1042F0008CA1822B808392B9EF8DF8A1908189A542
:1043000089238083EF8DF8A190818DA1892B8083F3
:10431000ED8DFE8D908188A58923808382E082B90E
:10432000EF8DF8A1908189A589238083EF8DF8A175
:1043300090818DA1892B8083ED8DFE8D90818CA144
:10434000892B808372B9EF8DF8A1908189A589238B
:104350008083EF8DF8A190818DA1892B8083ED8DD5
:10436000FE8D908188A58923808383E082B9EF8DBB
:10437000F8A1908189A589238083EF8DF8A1908190
:104380008DA1892B8083ED8DFE8D90818CA1892B51
:10439000808362B9EF8DF8A1908189A589238083FC
:1043A000EF8DF8A190818DA1892B8083ED8DFE8DFD
:1043B000908188A58923808386E082B9EF8DF8A15A
:1043C000908189A589238083EF8DF8A190818DA1AB
:1043D000892B8083ED8DFE8D90818CA1892B80832C
:1043E00052B9EF8DF8A1908189A589238083EF8D43
:1043F000F8A190818DA1892B8083ED8DFE8D908118
:1044000088A58923808387E082B9EF8DF8A1908108
:1044100089A589238083EF8DF8A190818DA1892BB7
:104420008083ED8DFE8D90818CA1892B808342B994
:10443000EF8DF8A1908189A589238083EF8DF8A164
:1044400090818DA1892B8083ED8DFE8D908188A533
:104450008923808382E21CC08250823008F045C0EC
:104460000A851B850150110928853985215031099C
:10447000CE010E947318EB8DFC8D90818FA1892352
:104480008083ED8DFE8D908188A5892380838CE2C9
:1044900082B9EF8DF8A1908189A589238083EF8D62
:1044A000F8A190818DA1892B8083ED8DFE8D908167
:1044B0008CA1892B8083E2B8EF8DF8A1908189A52A
:1044C00089238083EF8DF8A190818DA1892B808332
:1044D000F2B8EF8DF8A1908189A589238083EF8DB3
:1044E000F8A190818DA1892B8083EB8DFC8D90812B
:1044F0008BA1892B8083DF91CF911F910F91FF902A
:10450000EF900895EF92FF920F931F93CF93DF9355
:10451000EC010E944D14EB8DFC8D90818FA18923BD
:1045200080838A8D81115DC0ED89E150E33038F4DC
:10453000F0E0EE0FFF1FEE5EFD4F908101C090E3B3
:10454000ED8DFE8D208188A58223808312B8EF8DAA
:10455000F8A1208189A582238083EF8DF8A1208195
:104560008DA1822B808383E082B9EF8DF8A1208119
:1045700089A582238083EF8DF8A120818DA1822BD4
:104580008083ED8DFE8D20818CA1822B808380E144
:1045900082B9EF8DF8A1208189A582238083EF8DD8
:1045A000F8A120818DA1822B808392B9EF8DF8A193
:1045B000908189A589238083EF8DF8A190818DA1B9
:1045C000892B80830A851B8501501109288539852F
:1045D0002150310940E050E060E070E0CE010E94DF
:1045E00073188A8D8130A1F5ED89E150E33028F40C
:1045F000F0E0E15FFD4F908101C090E0ED8DFE8D18
:10460000208188A58223808386E182B9EF8DF8A17D
:10461000208189A582238083EF8DF8A120818DA13F
:10462000822B8083ED8DFE8D20818CA1822B808357
:1046300092B9EF8DF8A1908189A589238083EF8DB0
:10464000F8A190818DA1892B8083CE010E94BD1796
:104650008A8D823009F049C08D89813071F050F027
:10466000823029F0833059F458E2E52E08C068E41E
:10467000E62E05C048E8E42E02C038EEE32EED8DAC
:10468000FE8D908188A58923808386E382B9EF8D92
:10469000F8A1908189A589238083EF8DF8A190816D
:1046A0008DA1892B8083ED8DFE8D90818CA1892B2E
:1046B0008083E2B8EF8DF8A1908189A5892380835A
:1046C000EF8DF8A190818DA1892B80830A851B85B0
:1046D00001501109288539852150310940E050E009
:1046E00060E070E0CE010E9473188A8D833009F07B
:1046F00048C08D89813069F048F0823029F08330DC
:1047000051F420E6F22E07C0F12C05C090ECF92EF2
:1047100002C080EAF82EED8DFE8D908188A5892358
:10472000808386E382B9EF8DF8A1908189A58923E2
:104730008083EF8DF8A190818DA1892B8083ED8DF1
:10474000FE8D90818CA1892B8083F2B8EF8DF8A12A
:10475000908189A589238083EF8DF8A190818DA117
:10476000892B80830A851B8501501109288539858D
:104770002150310940E050E060E070E0CE010E943D
:104780007318DF91CF911F910F91FF90EF900895D3
:104790001F920F920FB60F9211240BB60F922F9308
:1047A0003F934F935F936F937F938F939F93AF93B9
:1047B000BF93EF93FF9383E19DE0D7DBFF91EF91F0
:1047C000BF91AF919F918F917F916F915F914F9129
:1047D0003F912F910F900BBE0F900FBE0F901F9027
:1047E00018951F920F920FB60F9211240BB60F92CD
:1047F0002F938F939F93EF93FF93E091230DF0916D
:10480000240D8081E091290DF0912A0D82FD12C0C6
:10481000908180912C0D8F5F8F7320912D0D8217C9
:1048200051F0E0912C0DF0E0ED5EF24F958F80930A
:104830002C0D01C08081FF91EF919F918F912F915D
:104840000F900BBE0F900FBE0F901F901895CF9238
:10485000DF92EF92FF92FC01A38DB48D9C9187A112
:1048600089238C93A58DB68D9C9180A589238C93EB
:1048700062B9A78DB0A19C9181A589238C93A78D46
:10488000B0A19C9185A1892B8C93A58DB68D9C910F
:1048900084A1892B8C9383E290E0DC011197F1F7DE
:1048A000C52EDD24EE24FF24C2B8A78DB0A17C91D3
:1048B00061A567236C93A78DB0A17C9165A1672B3F
:1048C0006C93DC011197F1F76A01EE24FF24C2B862
:1048D000A78DB0A17C9161A567236C93A78DB0A132
:1048E0007C9165A1672B6C93DC011197F1F7C32EC6
:1048F000D42EE52EFF24C2B8A78DB0A17C9161A56E
:1049000067236C93A78DB0A17C9165A1672B6C93F5
:104910000197F1F722B9A78DB0A19C9181A58923B8
:104920008C93A78DB0A19C9185A1892B8C93A38D8D
:10493000B48D9C9183A1892B8C93FF90EF90DF9095
:10494000CF9008952F923F924F925F926F927F92F5
:104950008F929F92AF92BF92CF92DF92EF92FF928F
:104960000F931F93CF93DF93CDB7DEB76B970FB63F
:10497000F894DEBF0FBECDBF9B8F8A8F5B011A01FB
:10498000D22E1F830E833701C982DC0158962D91E8
:104990003C9159972115310509F0E6C018968D9183
:1049A0009C911997681779070CF0CDC11A968D91D3
:1049B0009C911B97481759070CF0C5C18C2C912C62
:1049C000FB0126E0C29EE00DF11D1124FB87EA8762
:1049D0001E161F060CF0B7C1A40183E0440F551F3B
:1049E0008A95E1F75D874C87CA01820D931D1816E1
:1049F00019060CF0A8C157968C91811104C05FEA8A
:104A00005D1508F4D394AA8DBB8DED91FC9111979F
:104A10000284F385E02DCD011995B5E0DB9EC00140
:104A20001124F5013596FF87EE87BB82AA82250106
:104A30009C012A193B09398B288BA101485F5F4FE4
:104A40005B8B4A8BE889F989E40DF51DE259FD4D30
:104A50005491588761013D822C82888580FF13C064
:104A6000AA8DBB8DED91FC91B981B13031F40484F4
:104A7000F585E02D2E813F8116C00684F785E02D57
:104A8000EE80FF801AC0EE81FF81E615F705F1F098
:104A9000AA8DBB8DED91FC91B981B13051F40484A4
:104AA000F585E02D9301A601B2018A8D9B8D1995A4
:104AB0000DC00684F785E02D7301840194014C81BB
:104AC0005D816A817B818A8D9B8D1995E885E6954C
:104AD000E887FFEFCF1ADF0A2C813D81280D391DB1
:104AE0003D832C834A895B89C416D50609F0B5CF6E
:104AF0005FEF451A550A8A819B81880D991D9B831A
:104B00008A83AE85BF854A165B0609F09BCFEE818E
:104B1000FF81E615F70509F4F4C0EA8DFB8DA0814D
:104B2000B181F981F13079F4B5016B5F7F4F509617
:104B3000ED91FC915197830128E030E0A1018A8D2D
:104B40009B8D1995DEC06A857B85681979091E964B
:104B5000ED91FC911F9773010C851D859401A101B6
:104B60008A8D9B8D1995CDC0F9013496E491DE1A9A
:104B7000F901329685919491B7E0DB9E800D911DED
:104B80001124F901259134913B8B2A8BFC0125914D
:104B900034912901FC013296C490319634913E87BC
:104BA000329614913196D4904981423058F0612E5A
:104BB000012E000C77088D2D0D2C000C990B998778
:104BC000888704C019861886612C712CAA8DBB8D2C
:104BD000ED91FC9111970284F385E02DCD0119959B
:104BE000B9818B2E912C689CC001699C900D789C9A
:104BF000900D1124FC01EA0DFB1DFD87EC871A8244
:104C0000712C612CE12F110FFF0B95012E0F3F1F0F
:104C10003B872A87AC0CB11CA5014E0F5F1F5F8B31
:104C20004E8BC1018D0D911DD7FC9A95998F888F60
:104C30009E85691608F065C0862D90E048855985E7
:104C4000480F591F489D9001499D300D589D300DCA
:104C50001124D101A20FB31FB98BA88BEC85FD8560
:104C6000FD83EC83AA84BB84DA80FA85DF1A288D61
:104C7000398D280F391F3D8B2C8B8D2D8A0D4E8938
:104C80005F89A416B506C1F1877041F4C20101968F
:104C9000EA89FB89E40DF51D74902C0177FE21C093
:104CA000AA8DBB8DED91FC91B981B13061F4048482
:104CB000F585E02D2E813F814C895D89B5018A8D76
:104CC0009B8D19950EC00684F785E02DEE80FF8040
:104CD00084019401488959896C817D818A8D9B8DDD
:104CE0001995770CEFEFAE1ABE0A2C813D81280D85
:104CF000391D3D832C83C1CF3A813C0D3A836394A7
:104D000097CFAA8DBB8DED91FC9111970688F789FD
:104D1000E02DCD016B960FB6F894DEBF0FBECDBF70
:104D2000DF91CF911F910F91FF90EF90DF90CF9087
:104D3000BF90AF909F908F907F906F905F904F90BB
:104D40003F902F9019946B960FB6F894DEBF0FBE6C
:104D5000CDBFDF91CF911F910F91FF90EF90DF902A
:104D6000CF90BF90AF909F908F907F906F905F900B
:104D70004F903F902F900895362F90E0FC01E85D12
:104D8000FD4D4491FC01E857F84D2491FC01E85198
:104D9000F84D9491992309F46CC0442309F455C04B
:104DA00050E0FA013197E231F10508F04EC0882752
:104DB000EE58FF4F8F4F0C942231809180008F77F7
:104DC00007C0809180008F7D03C080918000877F25
:104DD000809380003AC084B58F7702C084B58F7D00
:104DE00084BD33C08091B0008F7703C08091B00044
:104DF0008F7D8093B00029C0809190008F7707C08D
:104E0000809190008F7D03C080919000877F809378
:104E100090001BC08091A0008F7707C08091A000F8
:104E20008F7D03C08091A000877F8093A0000DC07C
:104E3000809120018F7707C0809120018F7D03C072
:104E400080912001877F80932001E92FF0E0EE0F11
:104E5000FF1FE253F84DA591B4919FB7F89431111B
:104E600004C08C912095282302C0EC912E2B2C930A
:104E70009FBF08958F929F92AF92BF92CF92DF9281
:104E8000EF92FF926B017C010E94EF1D4B015C01D0
:104E9000C114D104E104F104F1F00E94EF1DDC0122
:104EA000CB0188199909AA09BB09883E9340A1053D
:104EB000B10570F321E0C21AD108E108F10888EECB
:104EC000880E83E0981EA11CB11CC114D104E1041A
:104ED000F10419F7DDCFFF90EF90DF90CF90BF90F6
:104EE000AF909F908F900895E091D10DF091D20DE9
:104EF00090818091D90D892B8083E091D50DF0911F
:104F0000D60D90818091DB0D892B8083E091D70DA8
:104F1000F091D80D90818091DC0D892B8083809158
:104F2000E10D882359F060E027DF62E070E080E067
:104F300090E0A0DF61E08091E10D1EDFE091D10DF6
:104F4000F091D20D90818091DD0D89238083E091D5
:104F5000D30DF091D40D90818091DE0D8923808353
:104F600012B8E091D50DF091D60D90818091DF0DB2
:104F700089238083E091D50DF091D60D90818091A9
:104F8000DB0D892B808383E0E091D50DF091D60D68
:104F900020819091DF0D92239083E091D50DF091C7
:104FA000D60D20819091DB0D922B9083815061F77B
:104FB000E091D10DF091D20D90818091D90D892B86
:104FC000808308957F928F929F92AF92BF92CF92EB
:104FD000DF92EF92FF920F931F93CF93DF93CDB7A2
:104FE000DEB768970FB6F894DEBF0FBECDBF7C0169
:104FF0008091B40D9091B50D892B39F0E091B00DF1
:10500000F091B10D8081811106C060E070E086EB07
:105010009DE00E94B31BF70184819581C69730F013
:1050200000E010E085E3C82ED12C14C0B701CE01FA
:1050300001960E94C71E65E07DE0CE01019614D363
:10504000BC0180EB9DE00E948B1ECE0101960E9468
:10505000C21E53C0F70124813581C901B6010E94E7
:105060000E31A901481B590B702F612F041715072A
:1050700020F50B5C1F4F9801472F562FB701CE012B
:1050800007960E94F41EBE01695F7F4FCE01019614
:105090000E94C71E65E07DE0CE010196E5D2BC010D
:1050A00080EB9DE00E948B1ECE0101960E94C21EE5
:1050B000CE0107960E94C21ECDCF892BF1F0B70119
:1050C000CE0107960E94F41EBE01695F7F4FCE019C
:1050D00001960E94C71E65E07DE0CE010196C4D214
:1050E000BC0180EB9DE00E948B1ECE0101960E94C8
:1050F000C21ECE0107960E94C21E60EB7DE0CE016B
:1051000007960E94C71E00E010E0E12CF12CA801D8
:105110008B859C850817190718F50F5F1F4F98019D
:10512000BE01695F7F4FCE0101960E94F41E8D8102
:105130009E81892B51F065E07DE089819A810E94F2
:105140004433DD24D394892B09F0D12CCE01019670
:105150000E94C21EDD20D9F2FFEFEF1AFF0AD7CF5F
:10516000CE0107960E94C21E8701015011098FE1EE
:10517000E816F1040CF442C065E07DE0CE01019632
:105180000E94E01EE090B40DF090B50DE114F10422
:1051900079F1C090B00DD090B10D69817A81C601CE
:1051A0000E946333009721F0BC016C197D0902C095
:1051B0006FEF7FEF6F5F7F4FD9F0E616F70608F4C9
:1051C000B701A701461B570B5093B50D4093B40D83
:1051D0006C0D7D1DC6010E945433E091B00DF0911D
:1051E000B10D8091B40D9091B50DE80FF91F1082AB
:1051F000CE0101960E94C21E7801B6CF8FEF9FEFBD
:105200009093C90D8093C80D9093C70D8093C60DE0
:1052100068E07DE0CE0143960E94E01E0F3FEFEF75
:105220001E0709F470C060EB7DE0CE010D960E9470
:10523000C71EE12CF12C912CA12CC12CD12C7E2C41
:105240008F2C89899A89E816F906B8F5FFEFEF1ACD
:10525000FF0A9701472D582DBE01635F7F4FCE0196
:1052600001960E94F41E8D819E81892B51F065E08C
:105270007DE089819A810E944433BB24B394892BB9
:1052800009F0B12CCE0101960E94C21EBB20B9F2DA
:10529000C60101960C151D0521F09E2CAF2C6C014A
:1052A000CECF272D382D492D5A2DBE01635F7F4F5C
:1052B000CE0107960E94F41E06C068E07DE0CE0194
:1052C00007960E94E01EBE01695F7F4FCE010196E6
:1052D0000E94C71E67E07DE0CE010196C5D1BC01EA
:1052E000CE0143960E948B1ECE0101960E94C21EE3
:1052F000CE0107960E94C21ECE010D960E94C21ECC
:10530000015011098BCF81E08093CA0D1092C30D1B
:105310001092C20D1092C50D1092C40D60E070E0A5
:1053200086EB9DE00E94B31B4F89588D6B897C8969
:1053300086EB9DE00E94451FCE0143960E94C21E4F
:1053400068960FB6F894DEBF0FBECDBFDF91CF9148
:105350001F910F91FF90EF90DF90CF90BF90AF9093
:105360009F908F907F9008951F93CF93DF93FC01C0
:10537000A38DB48D9C9187A189238C93A58DB68D27
:105380009C9180A589238C93828D823091F081112C
:105390000EC012B8A78DB0A19C9181A589238C93D2
:1053A000A78DB0A19C9185A1892B8C9304C08330DB
:1053B00011F48CE201C082E282B9A78DB0A19C9168
:1053C00081A589238C93A78DB0A19C9185A1892B60
:1053D0008C93A58DB68D9C9184A1892B8C9372B9E9
:1053E000A78DB0A19C9181A589238C93A78DB0A195
:1053F0009C9185A1892B8C9362B9A78DB0A19C91BA
:1054000081A589238C93A78DB0A19C9185A1892B1F
:105410008C932150310941095109DA01C90136E063
:10542000B695A795979587953A95D1F77613F0C0DD
:10543000019708F465C060E1A78DB0A1CC9171A57A
:105440007C237C93A78DB0A1CC9175A17C2B7C9300
:10545000A78DB0A1CC9171A57C237C93A78DB0A121
:10546000CC9175A17C2B7C93A78DB0A1CC9171A51B
:105470007C237C93A78DB0A1CC9175A17C2B7C93D0
:10548000A78DB0A1CC9171A57C237C93A78DB0A1F1
:10549000CC9175A17C2B7C93A78DB0A1CC9171A5EB
:1054A0007C237C93A78DB0A1CC9175A17C2B7C93A0
:1054B000A78DB0A1CC9171A57C237C93A78DB0A1C1
:1054C000CC9175A17C2B7C93A78DB0A1CC9171A5BB
:1054D0007C237C93A78DB0A1CC9175A17C2B7C9370
:1054E000A78DB0A1CC9171A57C237C93A78DB0A191
:1054F000CC9175A17C2B7C93615009F09DCF98CF06
:105500002F73215008F4A6C0A78DB0A19C9181A54E
:1055100089238C93A78DB0A19C9185A1892B8C9315
:10552000A78DB0A19C9181A589238C93A78DB0A153
:105530009C9185A1892B8C93E4CF72B9C78DD0A1A2
:105540001881B1A5B123B883C78DD0A11881B5A1A9
:10555000B12BB88362B9C78DD0A11881B1A5B12391
:10556000B883C78DD0A11881B5A1B12BB88372B90A
:10557000C78DD0A11881B1A5B123B883C78DD0A1A3
:105580001881B5A1B12BB88362B9C78DD0A118819C
:10559000B1A5B123B883C78DD0A11881B5A1B12B16
:1055A000B88372B9C78DD0A11881B1A5B123B883D2
:1055B000C78DD0A11881B5A1B12BB88362B9C78DB1
:1055C000D0A11881B1A5B123B883C78DD0A118810E
:1055D000B5A1B12BB88372B9C78DD0A11881B1A57F
:1055E000B123B883C78DD0A11881B5A1B12BB883E1
:1055F00062B9C78DD0A11881B1A5B123B883C78D79
:10560000D0A11881B5A1B12BB883A15009F095CFD5
:10561000019710F0A0E191CF2F732150D8F072B90B
:10562000A78DB0A19C9181A589238C93A78DB0A152
:105630009C9185A1892B8C9362B9A78DB0A19C9177
:1056400081A589238C93A78DB0A19C9185A1892BDD
:105650008C93E3CFA38DB48D9C9183A1892B8C93E4
:10566000DF91CF911F910895CF93DF93EC016115E6
:10567000710561F0FB0101900020E9F73197AF015E
:10568000461B570B0E945E1E811103C0CE010E9473
:10569000911ECE01DF91CF91089580EB9DE00C9497
:1056A000C21ECF93DF9300D000D0CDB7DEB7789481
:1056B00084B5826084BD84B5816084BD85B5826017
:1056C00085BD85B5816085BD80916E0081608093C8
:1056D0006E00109281008091810082608093810031
:1056E0008091810081608093810080918000816041
:1056F000809380008091B10084608093B10080919C
:10570000B00081608093B0008091910082608093AE
:105710009100809191008160809391008091900030
:105720008160809390008091A10082608093A100AD
:105730008091A10081608093A1008091A000816090
:105740008093A0008091210182608093210180914B
:1057500021018160809321018091200181608093EB
:10576000200180917A00846080937A0080917A0091
:10577000826080937A0080917A00816080937A00C1
:1057800080917A00806880937A001092C100E09145
:10579000230DF091240D12E01083E0911F0DF09184
:1057A000200D1082E091210DF091220D8FEC80836D
:1057B00010922B0DE091270DF091280D86E080834B
:1057C000E091250DF091260D808180618083E0912C
:1057D000250DF091260D808188608083E091250D54
:1057E000F091260D808180688083E091250DF091F5
:1057F000260D80818F7D808377DB76DB68EC70E01F
:1058000080E090E037DB1093D00DE091D10DF09166
:10581000D20D90818091DD0D89238083E091D30D9D
:10582000F091D40D90818091DE0D8923808381E0F9
:1058300082B9E091D50DF091D60D90818091DF0D68
:1058400089238083E091D50DF091D60D90818091D0
:10585000DB0D892B8083E091D30DF091D40D9081E5
:105860008091DA0D892B808312B8E091D50DF091EB
:10587000D60D90818091DF0D89238083E091D50D35
:10588000F091D60D90818091DB0D892B808362E3AE
:1058900070E080E090E0EEDAE091D30DF091D40D6D
:1058A00090818091DE0D8923808388E282B9E09126
:1058B000D50DF091D60D90818091DF0D89238083E5
:1058C000E091D50DF091D60D90818091DB0D892B63
:1058D0008083E091D30DF091D40D90818091DA0D09
:1058E000892B808312B8E091D50DF091D60D90816F
:1058F0008091DF0D89238083E091D50DF091D60D45
:1059000090818091DB0D892B8083E091D30DF09104
:10591000D40D90818091DE0D8923808390EC92B923
:10592000E091D50DF091D60D20818091DF0D82237D
:105930008083E091D50DF091D60D20818091DB0D13
:10594000822B8083E091D30DF091D40D2081809142
:10595000DA0D822B808383E282B9E091D50DF0913C
:10596000D60D20818091DF0D82238083E091D50DBB
:10597000F091D60D20818091DB0D822B8083E09108
:10598000D30DF091D40D20818091DE0D8223808390
:1059900081EC82B9E091D50DF091D60D20818091F6
:1059A000DF0D82238083E091D50DF091D60D20810B
:1059B0008091DB0D822B8083E091D30DF091D40D8B
:1059C00020818091DA0D822B808380E182B9E09181
:1059D000D50DF091D60D20818091DF0D822380833B
:1059E000E091D50DF091D60D20818091DB0D822BB9
:1059F0008083E091D30DF091D40D20818091DE0D54
:105A00008223808312B8E091D50DF091D60D2081CC
:105A10008091DF0D82238083E091D50DF091D60D2A
:105A200020818091DB0D822B808385EC82B9E0910F
:105A3000D50DF091D60D20818091DF0D82238083DA
:105A4000E091D50DF091D60D20818091DB0D822B58
:105A50008083E091D30DF091D40D20818091DA0DF7
:105A6000822B80832BE222B9E091D50DF091D60DE7
:105A700030818091DF0D83238083E091D50DF091FB
:105A8000D60D30818091DB0D832B808322B9E0918C
:105A9000D50DF091D60D20818091DF0D822380837A
:105AA000E091D50DF091D60D20818091DB0D822BF8
:105AB0008083E091D30DF091D40D20818091DE0D93
:105AC0008223808387EC82B9E091D50DF091D60DC9
:105AD00020818091DF0D82238083E091D50DF091AC
:105AE000D60D20818091DB0D822B8083E091D30D38
:105AF000F091D40D20818091DA0D822B808392B9B0
:105B0000E091D50DF091D60D90818091DF0D892324
:105B10008083E091D50DF091D60D90818091DB0DC1
:105B2000892B8083E091D30DF091D40D90818091E9
:105B3000DE0D8923808386E382B9E091D50DF09153
:105B4000D60D90818091DF0D89238083E091D50D62
:105B5000F091D60D90818091DB0D892B8083E091AF
:105B6000D30DF091D40D90818091DA0D892B808333
:105B700088E882B9E091D50DF091D60D90818091A1
:105B8000DF0D89238083E091D50DF091D60D9081B2
:105B90008091DB0D892B8083E091D30DF091D40DA2
:105BA00090818091DE0D892380838AE382B9E09120
:105BB000D50DF091D60D90818091DF0D89238083E2
:105BC000E091D50DF091D60D90818091DB0D892B60
:105BD0008083E091D30DF091D40D90818091DA0D06
:105BE000892B808385E582B9E091D50DF091D60DA2
:105BF00090818091DF0D89238083E091D50DF09114
:105C0000D60D90818091DB0D892B8083E091D30D9F
:105C1000F091D40D90818091DE0D8923808312B89C
:105C2000E091D50DF091D60D90818091DF0D892303
:105C30008083E091D50DF091D60D90818091DB0DA0
:105C4000892B808381EB82B9E091D50DF091D60D3F
:105C500090818091DF0D89238083E091D50DF091B3
:105C6000D60D90818091DB0D892B8083E091D30D3F
:105C7000F091D40D90818091DA0D892B808312B838
:105C8000E091D50DF091D60D90818091DF0D8923A3
:105C90008083E091D50DF091D60D90818091DB0D40
:105CA000892B80838BE182B9E091D50DF091D60DDF
:105CB00090818091DF0D89238083E091D50DF09153
:105CC000D60D90818091DB0D892B8083E091D30DDF
:105CD000F091D40D90818091DE0D8923808387EB34
:105CE00082B9E091D50DF091D60D90818091DF0DB4
:105CF00089238083E091D50DF091D60D908180911C
:105D0000DB0D892B8083E091D30DF091D40D908130
:105D10008091DA0D892B808387E082B9E091D50DDF
:105D2000F091D60D90818091DF0D89238083E091E1
:105D3000D50DF091D60D90818091DB0D892B80835C
:105D4000E091D30DF091D40D90818091DE0D8923E7
:105D5000808381E182B9E091D50DF091D60D9081DB
:105D60008091DF0D89238083E091D50DF091D60DD0
:105D700090818091DB0D892B8083E091D30DF09190
:105D8000D40D90818091DA0D892B808312B8E09137
:105D9000D50DF091D60D90818091DF0D8923808300
:105DA000E091D50DF091D60D90818091DB0D892B7E
:105DB000808366E970E080E090E05CD8E091D30DEC
:105DC000F091D40D90818091DE0D8923808389E24A
:105DD00082B9E091D50DF091D60D90818091DF0DC3
:105DE00089238083E091D50DF091D60D908180912B
:105DF000DB0D892B8083E091D30DF091D40D908140
:105E00008091DA0D892B808312B8E091D50DF09145
:105E1000D60D90818091DF0D89238083E091D50D8F
:105E2000F091D60D90818091DB0D892B808364EFFA
:105E300071E080E090E01ED80FE311E02FEE30E03B
:105E400040E050E060E070E086EB9DE00E94731857
:105E500061E086EB9DE00E9482226FEF7FEF86EB90
:105E60009DE00E94B31BC12CD12CB12C9EE0E92EE9
:105E7000F12C00E010E0C80187709927892B11F000
:105E8000B6940BC0F80183E0F595E7958A95E1F7A4
:105E9000EC0DFD1DE85FFE4FB490B0FE08C020EE93
:105EA00037E0A701B80186EB9DE00E942B160F5F3B
:105EB0001F4F003481E01807F1F68FEFE81AF80A57
:105EC00088E2C80ED11C82EEE816F10491F668E86B
:105ED00073E180E090E00E943A2760E070E086EB9A
:105EE0009DE00E94B31B66E572E0CE0101960E9420
:105EF000E01ECE01019666D8CE0101960E94C21E18
:105F000068EE73E080E090E00E943A276EE672E06F
:105F1000CE0101960E94E01ECE01019653D8CE011B
:105F200001960E94C21E62EC74E0CE0101960E94AE
:105F3000E01ECE01019646D8CE0101960E94C21EF7
:105F400060E976E0CE0101960E94E01ECE01019646
:105F500039D8CE0101960E94C21E40E050E068E0B0
:105F60007DE080EB9DE00E94A31E67EE77E0CE010E
:105F700001960E94E01ECE01019624D8CE01019622
:105F80000E94C21E66E079E0CE0101960E94E01EEA
:105F9000CE01019617D8CE0101960E94C21E68EE6E
:105FA00073E080E090E00E943A276FEC7CE0CE0145
:105FB00001960E94E01ECE01019604D8CE01019602
:105FC0000E94C21E10E060E0812F0E94BC261F5F6D
:105FD0001631C9F710E260E0812F0E94BC261F5FD6
:105FE0001633C9F70E944420FDCF90E0FC01E8572A
:105FF000F84D2491FC01E851F84D8491882399F0E3
:1060000090E0880F991FFC01E259F84DA591B491D9
:10601000FC01E253F84D859194918FB7F894EC917F
:10602000E22BEC938FBF0895BF92CF92DF92EF9255
:10603000FF920F931F93CF93DF93E3E1FDE0138271
:10604000128288EE93E0A0E0B0E084839583A6837B
:10605000B7838CE192E09183808385EC90E0958713
:10606000848784EC90E09787868780EC90E0918B22
:10607000808B81EC90E0938B828B82EC90E0958B0F
:10608000848B86EC90E0978B868B118E128E138E0C
:10609000148EC6EBDDE01B821A8280EFE82EF12C15
:1060A000FD82EC8200E411E01F830E83F986E8860E
:1060B0001B870A871D8A1D861C861F861E86BB2499
:1060C000B394BC8ACC24CA94DC2CDB8ACA8AD98AD1
:1060D000C88ABE8A1F8A198E188E8EE292E0998332
:1060E000888386E38BA7E1E2F8E2E491F0E0EE0F2B
:1060F000FF1FE253F84DA591B491BC8FAB8FE0E246
:10610000F8E2E491F0E0EE0FFF1FE253F84D8591C5
:1061100094919E8F8D8FEFE1F8E2E491F0E0EE0F25
:10612000FF1FE253F84D8591949198A38F8FEEE174
:10613000F8E2E491F0E0EE0FFF1FE253F84D859195
:1061400094919AA389A3E1ECF7E234913BA3E0ECAC
:10615000F7E224912CA3EFEBF7E294919DA3EEEBF1
:10616000F7E284918EA3432F40954FA3E22FE09551
:10617000E8A7E92FE095E9A7E82FE095EAA7EC91D9
:10618000E32BEC93ED8DFE8D90818CA1892B808388
:10619000EF8DF8A190818DA1892B8083E9A1FAA1CF
:1061A00090818EA1892B808389E31FDF88E31DDF27
:1061B00087E31BDF86E319DF61E086E30E94BC26EC
:1061C00086E313DF8FEF81B91D8A1D861C861F862B
:1061D0001E86BC8AD98AC88AF986E8861B870A8700
:1061E00068E07DE080EB9DE0DF91CF911F910F9102
:1061F000FF90EF90DF90CF90BF900C94E01EA29F95
:10620000B001B39FC001A39F700D811D1124911D8A
:10621000B29F700D811D1124911D0895AA1BBB1BF7
:1062200051E107C0AA1FBB1FA617B70710F0A61B96
:10623000B70B881F991F5A95A9F780959095BC01B7
:10624000CD010895EE0FFF1F881F8BBF0790F691B9
:10625000E02D1994D4DF332312F48A1B9B0B01C069
:10626000CEDFB7FF0895821B930B08950F931F9302
:10627000CF93DF938230910510F482E090E0E091BB
:10628000E40DF091E50D20E030E0A0E0B0E03097C3
:1062900019F1408151810281138148175907C8F0D3
:1062A0008417950769F4109731F012960C931297A2
:1062B00013961C9327C00093E40D1093E50D22C0A4
:1062C0002115310519F04217530718F49A01BD0141
:1062D000EF01DF01F801DBCF21153105F9F0281BB3
:1062E000390B2430310580F48A819B816115710559
:1062F00021F0FB019383828304C09093E50D80938A
:10630000E40DFE01329644C0FE01E20FF31F8193BB
:10631000919322503109398328833AC02091E20DAC
:106320003091E30D232B41F42091020230910302BE
:106330003093E30D2093E20D209100023091010291
:106340002115310541F42DB73EB74091040250911B
:106350000502241B350BE091E20DF091E30DE217ED
:10636000F307A0F42E1B3F0B2817390778F0AC0178
:106370004E5F5F4F2417350748F04E0F5F1F509355
:10638000E30D4093E20D8193919302C0E0E0F0E0D1
:10639000CF01DF91CF911F910F910895CF93DF939C
:1063A000009709F481C0FC01329713821282A091F8
:1063B000E40DB091E50D109781F420813181820FB9
:1063C000931F2091E20D3091E30D2817390751F505
:1063D000F093E30DE093E20D67C0ED0120E030E0C3
:1063E000CE17DF0740F44A815B819E0141155105BC
:1063F000F1F0EA01F5CFD383C28340815181840F4C
:10640000951FC817D90759F488819981840F951F62
:106410000296918380838A819B8193838283211555
:10642000310529F4F093E50DE093E40D3DC0E90159
:10643000FB83EA8349915991C40FD51FEC17FD07DF
:1064400061F480819181840F951F0296E9019983FF
:106450008883828193819B838A83E0E0F0E01296B7
:106460008D919C911397009719F0FD01DC01F7CFF6
:106470008D919C9111979D012E5F3F4F820F931F2D
:106480002091E20D3091E30D2817390769F4309718
:1064900029F41092E50D1092E40D02C013821282CD
:1064A000B093E30DA093E20DDF91CF9108956F9229
:1064B0007F928F929F92AF92BF92CF92DF92EF9294
:1064C000FF920F931F93CF93DF93009781F4CB013B
:1064D000DF91CF911F910F91FF90EF90DF90CF90C0
:1064E000BF90AF909F908F907F906F90BFCEFC0138
:1064F000E60FF71F9C0122503109E217F30708F459
:10650000A5C0EC01D9010D911C9111970617170731
:10651000A8F00530110508F497C0C8010497861744
:10652000970708F491C002501109061B170B01933D
:1065300011936D937C93CF0131DF86C05B01A01A6C
:10654000B10A4C01800E911EA091E40DB091E50DB1
:10655000612C712CE12CF12C109709F446C08D911F
:106560009C911197A815B905B1F56C0142E0C40ED4
:10657000D11CCA14DB0478F14C018A189B08640111
:1065800042E0C40ED11C1296BC9012971396AC91A7
:10659000B5E0CB16D10440F0B282A3839182808211
:1065A000D9016D937C9309C00E5F1F4F800F911F1F
:1065B000F90191838083EB2DFA2FE114F10431F07E
:1065C000D7011396FC93EE9312973EC0F093E50D1E
:1065D000E093E40D39C06816790608F43C017D01AA
:1065E00012960D90BC91A02DB7CF8091E20D9091A5
:1065F000E30D88169906E1F466167706C8F48091D3
:10660000000290910102009741F48DB79EB740912E
:10661000040250910502841B950BE817F907B0F4AA
:10662000F093E30DE093E20DF901718360830CC0F8
:10663000CB011CDE7C01009749F0A801BE011BD0F4
:10664000CE01ACDEC70104C0CE0102C080E090E004
:10665000DF91CF911F910F91FF90EF90DF90CF903E
:10666000BF90AF909F908F907F906F90089581E042
:1066700090E0F89442C0FB01DC0102C001900D9251
:1066800041505040D8F70895FB01DC018D910190F5
:1066900080190110D9F3990B0895FB01DC010190D9
:1066A0000D920020E1F70895FB01DC0141505040BC
:1066B00048F001900D920020C9F701C01D92415091
:1066C0005040E0F70895FB0151915523A9F0BF0117
:1066D000DC014D9145174111E1F759F4CD010190CD
:1066E000002049F04D9140154111C9F3FB014111C2
:1066F000EFCF81E090E00197089514E1C8E1D4E183
:1067000000E005C0802FFE019DDD2196011DC931ED
:0C671000D10780E00807B1F7F894FFCF34
:10671C000000E60D800000003F013F01EFEF00603C
:10672C00C0A028100010181000000000D71F451F33
:10673C006F1F2320A01F7E1F921F00000000E71672
:10674C00451FE416E3167C2002162B1603161F16A3
:10675C0013163216021682224C14011D641D7A1C6B
:10676C00B31BC1146214426F6F74696E6720477259
:10677C0065656E686F7573654F532E2E2E005374BE
:10678C007566662E636F2E6E7A3A204C6174657353
:10679C007420627265616B696E67206E6577732019
:1067AC004E5A3B68747470733A2F2F7777772E7329
:1067BC00747566662E636F2E6E7A2F3B427265611E
:1067CC006B696E67206E65777320616E64207669E5
:1067DC0064656F73206F6620746F64617927732012
:1067EC006C6174657374206E6577732073746F724B
:1067FC006965732066726F6D2061726F756E6420AF
:10680C004E6577205A65616C616E642C20696E63ED
:10681C006C7564696E6720757020746F2064617488
:10682C006520776561746865722C20576F726C6493
:10683C002C2073706F72742C20627573696E657383
:10684C00732C20456E7465727461696E6D656E741F
:10685C002C202E2E2E3B4E6174696F6E616C20C203
:10686C00B720E2808E576F726C6420C2B720E28032
:10687C008E53706F727420C2B720E2808E53747581
:10688C006666204E6174696F6E3B546F7020737432
:10689C006F726965733B54696E7920746F776E20E3
:1068AC007374726164646C696E672073746174656F
:1068BC0020686967687761792070757368657320E3
:1068CC00666F7220736166657220737065656473A0
:1068DC003B53747566662E636F2E6E7AC2B7332087
:1068EC00686F7572732061676F3B576861742069BC
:1068FC0073207265616C6C792064726976696E675D
:10690C0020746865202776696C69666963617469AF
:10691C006F6E27206F66204D656768616E204D6134
:10692C00726B6C653F3B53747566662E636F2E6E8F
:10693C007AC2B73120686F75722061676F3B5374F0
:10694C00727567676C696E67204A756C69616E2039
:10695C00536176656120746F6C6420746F206C6574
:10696C0061766520546F756C6F6E20627920616E54
:10697C0067727920626F7373202D207265706F724D
:10698C00743B53747566662E636F2E6E7AC2B73283
:10699C0020686F7572732061676F3B4D6F72652055
:1069AC00666F722073747566663B576562207265FC
:1069BC0073756C74733B4E6174696F6E616C204EB1
:1069CC00657773207C2053747566662E636F2E6E0C
:1069DC007A0041626F757420312C3738302C30308E
:1069EC00302C30303020726573756C747320283005
:1069FC002E3734207365636F6E647329203B5365A7
:106A0C006172636820526573756C74733B57656271
:106A1C0020726573756C74733B576F726C64206F66
:106A2C00662057617263726166743B68747470732C
:106A3C003A2F2F776F726C646F6677617263726135
:106A4C0066742E636F6D2F3B4A6F696E2074686F8E
:106A5C007573616E6473206F66206D6967687479F5
:106A6C00206865726F657320696E20417A65726F5C
:106A7C0074682C206120776F726C64206F66206DB7
:106A8C006167696320616E64206C696D69746C6503
:106A9C00737320616476656E747572652E3B476501
:106AAC007474696E672053746172746564202D2050
:106ABC00576F5720C2B720E2808E457520C2B72091
:106ACC00E2808E426174746C6520666F7220417A2C
:106ADC0065726F746820C2B720E2808E4261747454
:106AEC006C6520666F7220417A65726F7468202D18
:106AFC00204D65646961202D20576F573B574F57C8
:106B0C002120496E7465726E6574204361626C65F8
:106B1C0020616E642050686F6E65202D2042756E6A
:106B2C00646C65206F666665727320616E64207399
:106B3C007570706F72743B68747470733A2F2F7722
:106B4C0077772E776F777761792E636F6D2F3B4553
:106B5C0078706C6F7265206F6666657273207769EA
:106B6C00746820574F572120496E7465726E657496
:106B7C002C204361626C6520545620616E64204861
:106B8C006F6D652050686F6E652E2046696E6420AF
:106B9C00746865206F6666657220616E642074008F
:106BAC0023696E636C756465203C737472696E67DF
:106BBC002E683E3B23696E636C756465203C636F85
:106BCC006E696F2E683E3B23696E636C756465203D
:106BDC003C63747970652E683E3B23696E636C75FB
:106BEC006465203C77696E646F77732E683E3B69F1
:106BFC006E74206D61696E28696E742061726763B2
:106C0C002C2063686172202A617267765B5D293B78
:106C1C007B3B636861722073656E747A7A5B5D3D51
:106C2C002248454C4C4F204920414D204120544591
:106C3C005854205343524F4C4C223B2020202020B0
:106C4C002020202020202020223B696E7420783BBD
:106C5C0020202020202020202020202020202F2F0A
:106C6C007370656369616C206469616C6F677565CD
:106C7C003B696E742073697A653B203B73697A6556
:106C8C003D7374726C656E2873656E7461293B205C
:106C9C002020666F7228783D303B783C73697A65AA
:106CAC003B782B2B293B202020207B2020203B20B5
:106CBC00202020202020536C656570283430293B1F
:106CCC002020202020202020207072696E746628DD
:106CDC00222563222C73656E74615B785D293B20E1
:106CEC002020207D3B2020202067657463682829A4
:106CFC003B202020207D00496E206D7920796F7516
:106D0C006E67657220616E64206D6F72652076759A
:106D1C006C6E657261626C65207965617273206D51
:106D2C0079206661746865722067617665206D658F
:106D3C0020736F6D6520616476696365207468618A
:106D4C00742049E280997665206265656E207475C1
:106D5C00726E696E67206F76657220696E206D7930
:106D6C00206D696E6420657665722073696E63654B
:106D7C002E20E280985768656E6576657220796F73
:106D8C0075206665656C206C696B6520637269742F
:106D9C006963697A696E6720616E79206F6E652C04
:106DAC00E2809920686520746F6C64206D652C20DE
:106DBC00E280986A7573742072656D656D62657298
:106DCC00207468617420616C6C2074686520706537
:106DDC006F706C6520696E207468697320776F72B0
:106DEC006C6420686176656EE280997420686164D9
:106DFC002074686520616476616E746167657320C8
:106E0C007468617420796F75E28099766520686189
:106E1C00642EE28099004865206469646E74207366
:106E2C00617920616E79206D6F72652062757420B6
:106E3C007765766520616C77617973206265656E24
:106E4C0020756E757375616C6C7920636F6D6D75E3
:106E5C006E6963617469766520696E206120726564
:106E6C00736572766564207761792C20616E64207D
:106E7C004920756E64657273746F6F6420746861F9
:106E8C0074206865206D65616E7420612067726581
:106E9C006174206465616C206D6F7265207468612B
:106EAC006E20746861742E20496E20636F6E73655A
:106EBC007175656E636520496D20696E636C696ED2
:106ECC00656420746F207265736572766520616CE1
:106EDC006C206A7564676D656E74732C2061206814
:106EEC0061626974207468617420686173206F70CA
:106EFC00656E6564207570206D616E7920637572A6
:106F0C00696F7573206E61747572657320746F2070
:106F1C006D6520616E6420616C736F206D616465BA
:106F2C00206D65207468652076696374696D206FC7
:106F3C0066206E6F742061206665772076657465B7
:106F4C0072616E20626F7265732E205468652061C9
:106F5C00626E6F726D616C206D696E642069732056
:106F6C00717569636B20746F20646574656374203C
:106F7C00616E642061747461636820697473656CFC
:106F8C006620746F2074686973207175616C697404
:106F9C0079207768656E2069742061707065617204
:106FAC007320696E2061206E6F726D616C2070654C
:106FBC0072736F6E2C20616E6420736F2069742065
:106FCC0063616D652061626F7574207468617420F3
:106FDC00696E20636F6C6C656765204920776173FF
:106FEC0020756E6A7573746C792061636375736553
:106FFC0064206F66206265696E67206120706F6C1B
:10700C006974696369616E2C20626563617573656F
:10701C0020492077617320707269767920746F2013
:10702C007468652073656372657420677269656640
:10703C0073206F662077696C642C20756E6B6E6F95
:10704C00776E206D656E2E204D6F7374206F6620E9
:10705C0074686520636F6E666964656E6365732022
:10706C007765726520756E736F756768742D6672BF
:10707C00657175656E746C79204920686176652040
:10708C00666569676E656420736C6565702C20702D
:10709C0072656F636375706174696F6E2C206F72AB
:1070AC00206120686F7374696C65206C65766974F7
:1070BC0079207768656E2049207265616C697A6504
:1070CC006420627920736F6D6520756E6D697374C1
:1070DC00616B61626C65207369676E2074686174A2
:1070EC0020616E20696E74696D61746520726576BD
:1070FC00656C6174696F6E20776173207175697648
:10710C006572696E67206F6E2074686520686F7297
:10711C00697A6F6E2D666F722074686520696E7463
:10712C00696D61746520726576656C6174696F6EEA
:10713C0073206F6620796F756E67206D656E206F9A
:10714C0072206174206C656173742074686520749E
:10715C0065726D7320696E20776869636820746846
:10716C0065792065787072657373207468656D201D
:10717C0061726520757375616C6C7920706C6167D8
:10718C00696172697374696320616E64206D6172E8
:10719C00726564206279206F6276696F75732073F3
:1071AC0075707072657373696F6E732E2052657390
:1071BC00657276696E67206A7564676D656E747347
:1071CC002069732061206D6174746572206F662074
:1071DC00696E66696E69746520686F70652E005BF8
:1071EC0020204F4B20205D20456E61626C696E67DC
:1071FC0020706F776572736176696E672066656162
:10720C0074757265732E2E2E2020202020202020B5
:0A721C0020202020003B000A0000A3
:020000023000CC
:10E000000D9489F10D94B2F10D94B2F10D94B2F129
:10E010000D94B2F10D94B2F10D94B2F10D94B2F1F0
:10E020000D94B2F10D94B2F10D94B2F10D94B2F1E0
:10E030000D94B2F10D94B2F10D94B2F10D94B2F1D0
:10E040000D94B2F10D94B2F10D94B2F10D94B2F1C0
:10E050000D94B2F10D94B2F10D94B2F10D94B2F1B0
:10E060000D94B2F10D94B2F10D94B2F10D94B2F1A0
:10E070000D94B2F10D94B2F10D94B2F10D94B2F190
:10E080000D94B2F10D94B2F10D94B2F10D94B2F180
:10E090000D94B2F10D94B2F10D94B2F10D94B2F170
:10E0A0000D94B2F10D94B2F10D94B2F10D94B2F160
:10E0B0000D94B2F10D94B2F10D94B2F10D94B2F150
:10E0C0000D94B2F10D94B2F10D94B2F10D94B2F140
:10E0D0000D94B2F10D94B2F10D94B2F10D94B2F130
:10E0E0000D94B2F141546D656761323536300041AF
:10E0F000726475696E6F206578706C6F72657220DE
:10E1000073746B3530305632206279204D4C530099
:10E11000426F6F746C6F616465723E004875683F52
:10E1200000436F6D70696C6564206F6E203D200048
:10E130004350552054797065202020203D20005FF9
:10E140005F4156525F415243485F5F3D2000415658
:10E1500052204C696243205665723D20004743437C
:10E160002056657273696F6E203D20004350552024
:10E1700049442020202020203D20004C6F7720663D
:10E18000757365202020203D20004869676820665F
:10E190007573652020203D200045787420667573D6
:10E1A00065202020203D20004C6F636B2066757336
:10E1B000652020203D20004D617220203720323024
:10E1C000313300312E362E3800342E332E350056A2
:10E1D00023202020414444522020206F7020636F70
:10E1E00064652020202020696E73747275637469E1
:10E1F0006F6E2061646472202020496E74657272B3
:10E20000757074006E6F20766563746F7200726A49
:10E210006D702020006A6D70200057686174207056
:10E220006F72743A00506F7274206E6F7420737541
:10E2300070706F72746564004D7573742062652030
:10E2400061206C6574746572002000577269747483
:10E25000696E672045450052656164696E672045B7
:10E26000450045452065727220636E743D00504F35
:10E27000525400303D5A65726F2061646472003FF1
:10E280003D43505520737461747300403D454550C3
:10E29000524F4D207465737400423D426C696E6B41
:10E2A000204C454400453D44756D70204545505215
:10E2B0004F4D00463D44756D7020464C415348001B
:10E2C000483D48656C70004C3D4C69737420492F83
:10E2D0004F20506F72747300513D51756974005234
:10E2E0003D44756D702052414D00563D73686F7707
:10E2F00020696E7465727275707420566563746FF0
:10E30000727300593D506F727420626C696E6B00BD
:10E310002A0011241FBECFEFD1E2DEBFCDBF01E046
:10E320000CBF12E0A0E0B2E0EEE1FDEF03E00BBFB6
:10E3300002C007900D92A030B107D9F712E0A0E01B
:10E34000B2E001C01D92AE30B107E1F70F9460F367
:10E350000D948DFE01E20EBF0FEF0DBF11241FBE05
:10E360000D9460F30D9400F020E030E040ED57E0B4
:10E3700005C0FA013197F1F72F5F3F4F2817390792
:10E38000C0F308959C01260F311DC901A0E0B0E043
:10E390002F5F3F4FABBFFC018791882361F08093D3
:10E3A000C6008091C00086FFFCCF8091C0008064D1
:10E3B0008093C000EACF08958DE08093C6008091DD
:10E3C000C00086FFFCCF8091C00080648093C000B5
:10E3D0008AE08093C6008091C00086FFFCCF8091C8
:10E3E000C00080648093C00008950F94C2F10F9420
:10E3F000DCF10895FC019081992359F09093C600B7
:10E400008091C00086FFFCCF8091C0008064809323
:10E41000C0003196992379F70895282F982F929567
:10E420009F70892F805D8A3308F0895F8093C600D2
:10E430008091C00086FFFCCF8091C00080648093F3
:10E44000C000822F8F70982F905D9A3308F0995FEB
:10E450009093C6008091C00086FFFCCF8091C000E1
:10E4600080648093C00008959C01FB01853691056E
:10E470001CF46330710594F0C90164E670E00F94F8
:10E480002EFE605D7F4F6093C6008091C00086FFC6
:10E49000FCCF8091C00080648093C0002B30310598
:10E4A00014F43297B4F0C90164E670E00F942EFEC4
:10E4B0006AE070E00F942EFE605D7F4F6093C600AF
:10E4C0008091C00086FFFCCF8091C0008064809363
:10E4D000C000C9016AE070E00F942EFEC0968093E0
:10E4E000C6008091C00086FFFCCF8091C000806490
:10E4F0008093C00008951F93182F8EE692EE60E07F
:10E500000F94C2F11093C6008091C00086FFFCCF2B
:10E510008091C00080648093C0000F94DCF11F9153
:10E5200008952F923F924F925F926F927F928F92B7
:10E530009F92AF92BF92CF92DF92EF92FF920F9392
:10E540001F93DF93CF93CDB7DEB762970FB6F894E2
:10E55000DEBF0FBECDBF382E622ECA01DB015C01CB
:10E560006D01772420E2222E2E010894411C511CBB
:10E570008BC081E0A81680E0B80681E0C80680E084
:10E58000D80628F0C601AA27BB270F940DF2BB2797
:10E59000AD2D9C2D8B2D0F940DF28A2D0F940DF225
:10E5A0002092C6008091C00086FFFCCF8091C00001
:10E5B00080648093C0009DE29093C6008091C0006B
:10E5C00086FFFCCF8091C00080648093C0002092C1
:10E5D000C6008091C00086FFFCCF8091C00080649F
:10E5E0008093C00019828601750188249924A1E0D6
:10E5F0003A1651F03A1620F0B2E03B1661F409C029
:10E600000BBFF701779007C0C7010F9477FE782EF4
:10E6100002C0F7017080872D0F940DF22092C60082
:10E620008091C00086FFFCCF8091C0008064809301
:10E63000C000872D8052F401EF70F0708F3520F408
:10E64000E40DF51D708204C0E40DF51D8EE280839B
:10E650000894E11CF11C011D111D0894811C911CE2
:10E6600090E18916910409F0C2CF80E190E0A0E02A
:10E67000B0E0A80EB91ECA1EDB1E198AC2010F9493
:10E68000FAF10F94DCF16A94662009F072CF629679
:10E690000FB6F894DEBF0FBECDBFCF91DF911F91B3
:10E6A0000F91FF90EF90DF90CF90BF90AF909F9031
:10E6B0008F907F906F905F904F903F902F90089534
:10E6C0002F923F924F925F926F927F928F929F9282
:10E6D000AF92BF92CF92DF92EF92FF920F931F9370
:10E6E000DF93CF93CDB7DEB7CD53D1400FB6F894BB
:10E6F000DEBF0FBECDBF01E20EBF0FEF0DBF94B75F
:10E70000F894A89514BE80916000886180936000A1
:10E7100010926000789493FF05C0E0910002F091A0
:10E7200001021995279A2F9A8091C00082608093E8
:10E73000C00080E18093C40088E18093C1000000A4
:10E74000EE24FF24870144E0A42EB12CCC24DD2448
:10E7500024C0C5010197F1F70894E11CF11C011DCB
:10E76000111D21E2E2162EE4F20620E0020720E06D
:10E77000120718F031E0C32ED12CC801B70127ECE5
:10E780003BE140E050E00F9441FE611571058105C9
:10E79000910519F485B1805885B98091C00087FD35
:10E7A00003C0C114D104A9F2A6014F5F5F4FC25E3E
:10E7B000DE4F59834883CE51D140C25EDE4F8881FF
:10E7C0009981CE51D140019711F00D9410FEC05D9A
:10E7D000DE4F19821882C053D14060E0C15DDE4F28
:10E7E0001882CF52D14088249924C35DDE4F19820C
:10E7F0001882CD52D140C05EDE4F188219821A8233
:10E800001B82C052D140CE5CDE4F188219821A8220
:10E810001B82C253D140EE24FF2487010BBFF701B6
:10E8200007911691C45CDE4F19830883CC53D14005
:10E830000D940BFEC25EDE4F28813981CE51D1404E
:10E840002130310509F52091C600C25EDE4F1982E4
:10E850001882CE51D14022C02F5F3F4F4F4F5F4FA4
:10E86000213082E138078AE7480780E0580780F0C6
:10E87000C45CDE4FE881F981CC53D140EF5FFF4F9C
:10E8800019F0EE27FF27099420E030E040E050E047
:10E890008091C00087FFE0CF2091C600C35DDE4FAE
:10E8A00048815981CD52D1404F5F5F4FC35DDE4FEC
:10E8B00059834883CD52D140213209F063C64A3092
:10E8C000510508F05FC60894811C911C53E0851621
:10E8D000910409F059C600E010E018C081E280936D
:10E8E000C6008091C00086FFFCCF8091C00080648C
:10E8F0008093C0002F5F3F4F2931310579F70F9486
:10E90000DCF10F5F1F4F0530110519F020E030E0FA
:10E91000E5CF10920A0210920B0210920C02109294
:10E920000D02109206021092070210920802109235
:10E930000902109202021092030210920402109235
:10E9400005028FEE90EE60E00F94F5F180E191EE1C
:10E9500060E00F94C2F18091C00087FFFCCF9091DE
:10E96000C600903608F09F759032B8F09093C600BC
:10E970008091C00086FFFCCF8091C00080648093AE
:10E98000C000A0E2A093C6008091C00086FFFCCF2B
:10E990008091C00080648093C000983409F4D7C18E
:10E9A0009934B8F4923409F459C1933458F490333B
:10E9B00019F1903308F4E3C59F33A1F1903409F0C5
:10E9C000DEC5BDC0953409F470C1963409F0D7C5D1
:10E9D00098C1923509F42BC2933538F49C3409F46C
:10E9E000F5C1913509F0CBC518C2963509F445C279
:10E9F000993509F0C4C567C483E792EE62E00F94CD
:10EA0000F5F110920602109207021092080210927D
:10EA1000090210920A0210920B0210920C0210923C
:10EA20000D0213C18FE792EE62E00F94F5F18FEEC5
:10EA300090EE60E00F94F5F181E291EE60E00F94CA
:10EA4000C2F187EB91EE60E00F94F5F180E391EE77
:10EA500060E00F94C2F184EE90EE60E00F94F5F167
:10EA60008FE391EE60E00F94C2F186E090E061E008
:10EA700070E00F9434F20F94DCF18DE591EE60E0DC
:10EA80000F94C2F189EC91EE60E00F94F5F18EE401
:10EA900091EE60E00F94C2F183EC91EE60E00F9490
:10EAA000F5F18CE691EE60E00F94C2F18EE10F94E7
:10EAB0000DF288E90F940DF281E00F940DF20F949E
:10EAC000DCF18BE791EE60E00F94C2F119E0E0E039
:10EAD000F0E010935700E4918E2F0F940DF20F94F5
:10EAE000DCF18AE891EE60E00F94C2F1E3E0F0E03F
:10EAF00010935700E4918E2F0F940DF20F94DCF1D8
:10EB000089E991EE60E00F94C2F1E2E0F0E0109349
:10EB10005700E4918E2F0F940DF20F94DCF188EAE8
:10EB200091EE60E00F94C2F1E1E0F0E01093570045
:10EB30001491812F0F940DF20F94DCF107CF8BE825
:10EB400092EE62E00F94F5F18BE492EE60E00F94A8
:10EB5000F5F10F94DCF100E010E019C0C8016F2D51
:10EB60000F947FFEFF2031F489E492EE60E00F9471
:10EB7000C2F10BC0F092C6008091C00086FFFCCFAE
:10EB80008091C00080648093C0000F5F1F4FC80158
:10EB900081519F41A0E0B0E0ABBFFC01F790BAE229
:10EBA000FB1621F0E2E000301E07C1F60F94DCF105
:10EBB0000F94DCF187E592EE60E00F94F5F10F948D
:10EBC000DCF1CC24DD2400E010E01EC0C8010F946D
:10EBD00077FEF82E882331F489E492EE60E00F94FA
:10EBE000C2F10BC08093C6008091C00086FFFCCFAD
:10EBF0008091C00080648093C000FE1419F00894D6
:10EC0000C11CD11C0F5F1F4FC80181519F41A0E063
:10EC1000B0E0ABBFFC01E790FAE2EF1621F022E092
:10EC20000030120799F60F94DCF10F94DCF182E6C4
:10EC300092EE60E00F94C2F1C60161E070E00F94C3
:10EC400034F20F94DCF10F94DCF110920202109276
:10EC50000302109204021092050278CE89E992EE26
:10EC600062E00F94F5F1279A2F9A16C02F9880E052
:10EC700090E0E0EDF7E03197F1F7019684369105E9
:10EC8000C1F72F9A80E090E0E0EDF7E03197F1F7DF
:10EC9000019684369105C1F78091C00087FFE6CFC9
:10ECA0008091C00087FFFCCF64C485EA92EE62E0E9
:10ECB0000F94F5F140910202509103026091040219
:10ECC0007091050281E020E10F9491F2809102029F
:10ECD00090910302A0910402B091050280509F4FD1
:10ECE000AF4FBF4F8093020290930302A0930402A0
:10ECF000B093050280509041A040B04008F426CE69
:10ED0000A4CF83EB92EE62E00F94F5F140910602FE
:10ED100050910702609108027091090280E020E1A1
:10ED20000F9491F28091060290910702A09108023F
:10ED3000B091090280509F4FAF4FBF4F80930602A2
:10ED400090930702A0930802B0930902FFCD80ECD4
:10ED500092EE62E00F94F5F183E792EE60E00F949B
:10ED6000F5F18FE792EE60E00F94F5F18BE892EE0B
:10ED700060E00F94F5F189E992EE60E00F94F5F10F
:10ED800085EA92EE60E00F94F5F183EB92EE60E09D
:10ED90000F94F5F180EC92EE60E00F94F5F187ECC2
:10EDA00092EE60E00F94F5F188ED92EE60E00F9442
:10EDB000F5F18FED92EE60E00F94F5F18AEE92EEB0
:10EDC00060E00F94F5F183E093EEBDCD87EC92EE19
:10EDD00062E00F94F5F181E40F947BF282E40F94EA
:10EDE0007BF283E40F947BF284E40F947BF285E45E
:10EDF0000F947BF286E40F947BF287E40F947BF20E
:10EE000088E40F947BF28AE40F947BF28BE40F94F6
:10EE10007BF28CE40F947BF299CD88ED92EE62E068
:10EE20000F94F5F1772473948824992409C48FED05
:10EE300092EE62E00F94F5F140910A0250910B02BC
:10EE400060910C0270910D0282E020E10F9491F22A
:10EE500080910A0290910B02A0910C02B0910D02D8
:10EE600080509F4FAF4FBF4F80930A0290930B0289
:10EE7000A0930C02B0930D0269CD8AEE92EE62E08F
:10EE80000F94F5F184EE90EE60E00F94F5F18FECC5
:10EE900091EE60E00F94F5F1662477244301CC5D98
:10EEA000DE4F19821882C452D140D401C301B695F5
:10EEB000A79597958795CA5DDE4F88839983AA8326
:10EEC000BB83C652D140CC5DDE4FA881B981C4520C
:10EED000D1401196CC5DDE4FB983A883C452D14096
:10EEE000CD0162E070E00F9434F2B0E2B093C6005E
:10EEF0008091C00086FFFCCF8091C0008064809329
:10EF0000C000EDE2E093C6008091C00086FFFCCF18
:10EF10008091C00080648093C000F0E2F093C6004E
:10EF20008091C00086FFFCCF8091C00080648093F8
:10EF3000C000CA5DDE4FE880F9800A811B81C6529D
:10EF4000D140BB27A12F902F8F2D0F940DF2CA5DBA
:10EF5000DE4F8881C652D1400F940DF2B0E2FB2EF5
:10EF6000F092C6008091C00086FFFCCF8091C00067
:10EF700080648093C0000DE30093C6008091C000C0
:10EF800086FFFCCF8091C00080648093C00010E2B7
:10EF90001093C6008091C00086FFFCCF8091C00016
:10EFA00080648093C0008BBEF3012791C65DDE4F65
:10EFB0002883CA52D140A22EBB24CC24DD2408943D
:10EFC000611C711C811C911C8BBEF3018791282E42
:10EFD0003324442455240894611C711C811C911C09
:10EFE0008BBEF3013791C55DDE4F3883CB52D140E4
:10EFF0000894611C711C811C911C8BBEF30147910C
:10F00000C45DDE4F4883CC52D140ADEFEA2EAFEF66
:10F01000FA2EAFEF0A2FAFEF1A2F6E0C7F1C801E57
:10F02000911E142D032DF22CEE24EA0CFB1C0C1D5A
:10F030001D1D0F940DF220E22093C6008091C000A8
:10F0400086FFFCCF8091C00080648093C000C65DC5
:10F05000DE4F8881CA52D1400F940DF230E23093D6
:10F06000C6008091C00086FFFCCF8091C000806404
:10F070008093C000C45DDE4F8881CC52D1400F9494
:10F080000DF240E24093C6008091C00086FFFCCFA5
:10F090008091C00080648093C000C55DDE4F888190
:10F0A000CB52D1400F940DF250E25093C6008091A4
:10F0B000C00086FFFCCF8091C00080648093C000B8
:10F0C0008FEFE8168FEFF80680E0080780E018075A
:10F0D00031F484E092EE60E00F94C2F1DFC0D80119
:10F0E000C7018070907CA070B0708050904CA040A0
:10F0F000B040D1F52FEF3FE340E050E0E222F322B1
:10F1000004231523CA5DDE4FA880B980CA80DB8046
:10F11000C652D140AE0CBF1CC01ED11EAA0CBB1CD7
:10F12000CC1CDD1C8EE092EE60E00F94C2F1BB2798
:10F13000A12F902F8F2D0F940DF28E2D0F940DF285
:10F1400030E23093C6008091C00086FFFCCF8091F2
:10F15000C00080648093C0004EE34093C60080915D
:10F16000C00086FFFCCF87C08EE09EEFA0E0B0E03D
:10F17000E822F9220A231B239CE0E91694E9F90608
:10F1800090E0090790E0190709F088C0C45DDE4FE0
:10F19000A881CC52D140EA2EFF2400E010E0102FCD
:10F1A0000F2DFE2CEE24C55DDE4FB881CB52D14031
:10F1B000EB0EF11C011D111DD601C501817090706F
:10F1C000A070B070DC0199278827E80EF91E0A1F8D
:10F1D0001B1F20EF30E040E050E0A222B322C42207
:10F1E000D52241E1AA0CBB1CCC1CDD1C4A95D1F7F1
:10F1F000EA0CFB1C0C1D1D1D81E090E0A0E0B0E0BE
:10F20000282239224A225B2235E1220C331C441C7D
:10F21000551C3A95D1F7E20CF31C041D151D57013E
:10F220006801AA0CBB1CCC1CDD1C85E192EE60E0E1
:10F230000F94C2F1C801AA27BB270F940DF2BB2778
:10F24000A12F902F8F2D0F940DF28E2D0F940DF274
:10F2500090E29093C6008091C00086FFFCCF809121
:10F26000C00080648093C000AEE3A093C60080918C
:10F27000C00086FFFCCF8091C00080648093C000F6
:10F28000C601AA27BB270F940DF2BB27AD2D9C2DDD
:10F290008B2D0F940DF28A2D0F940DF20F94DCF14B
:10F2A000CC5DDE4FE881F981C452D140F99709F471
:10F2B0004DCBF4E0EF2EF12C012D112D6E0C7F1CA7
:10F2C000801E911EF2CD83E093EE62E00F94F5F183
:10F2D0008AE192EE60E00F94C2F18091C00087FF56
:10F2E000FCCF1091C6001F751093C6008091C0001E
:10F2F00086FFFCCF8091C00080648093C0000F9493
:10F30000DCF1812F81548A3108F036C1163409F4BA
:10F3100095C0173490F4133409F44EC0143430F40B
:10F320001134F1F0123409F01DC130C0143409F465
:10F3300059C0153409F016C16BC01A3409F4C4C0A1
:10F340001B3438F4173409F48FC0183409F00AC19B
:10F35000A1C01B3409F4D2C01C3409F003C1E8C0B9
:10F360008FEF81B90DC082B1809582B980E090E0C5
:10F37000E0EDF7E03197F1F70196883C9105C1F790
:10F380008091C00087FFEFCF12B8EFC08FEF84B934
:10F390000DC085B1809585B980E090E0E0EDF7E0A3
:10F3A0003197F1F70196883C9105C1F78091C00033
:10F3B00087FFEFCF15B8D9C08FEF87B90DC088B1DF
:10F3C000809588B980E090E0E0EDF7E03197F1F7C3
:10F3D0000196883C9105C1F78091C00087FFEFCF6F
:10F3E00018B8C3C08FEF8AB90DC08BB180958BB9A7
:10F3F00080E090E0E0EDF7E03197F1F70196883C8E
:10F400009105C1F78091C00087FFEFCF1BB8ADC059
:10F410008FEF8DB90DC08EB180958EB980E090E0F0
:10F42000E0EDF7E03197F1F70196883C9105C1F7DF
:10F430008091C00087FFEFCF1EB897C08FEF80BBD1
:10F440000DC081B3809581BB80E090E0E0EDF7E0F6
:10F450003197F1F70196883C9105C1F78091C00082
:10F4600087FFEFCF11BA81C08FEF83BB0DC084B38C
:10F47000809584BB80E090E0E0EDF7E03197F1F714
:10F480000196883C9105C1F78091C00087FFEFCFBE
:10F4900014BA6BC08FEF809301010FC080910201FD
:10F4A00080958093020180E090E0E0EDF7E03197F5
:10F4B000F1F70196883C9105C1F78091C00087FF64
:10F4C000EDCF1092020151C08FEF809304010FC065
:10F4D0008091050180958093050180E090E0E0ED4A
:10F4E000F7E03197F1F70196883C9105C1F78091DB
:10F4F000C00087FFEDCF1092050137C08FEF8093DA
:10F5000007010FC08091080180958093080180E079
:10F5100090E0E0EDF7E03197F1F70196883C910536
:10F52000C1F78091C00087FFEDCF109208011DC088
:10F530008FEF80930A010FC080910B01809580931B
:10F540000B0180E090E0E0EDF7E03197F1F70196F4
:10F55000883C9105C1F78091C00087FFEDCF1092E4
:10F560000B0103C085E292EEEEC98091C00087FFD7
:10F57000FCCF8091C600EAC988E392EEE4C98CE131
:10F5800091EEE1C988249924933011F1943028F444
:10F59000913089F09230B8F408C0953061F195301F
:10F5A000F0F0963009F048C043C02B3109F042C951
:10F5B00091E06BE13FC96227C15DDE4F2883CF52E6
:10F5C000D14092E037C9B22FA0E0622793E032C960
:10F5D000822F90E0A82BB92B622794E02BC92E3004
:10F5E00009F039C3622795E0C05DDE4F19821882A9
:10F5F000C053D1401FC9E1E0F0E0EC0FFD1FC05D3A
:10F60000DE4F08811981C053D140E00FF11F2083E4
:10F610000F5F1F4FC05DDE4F19830883C053D14079
:10F6200062270A171B0709F005C9D80196E002C92D
:10F63000261709F010C303C0973009F0FBC87724E0
:10F640009981933109F412C19431C8F4963009F4C8
:10F65000D8C0973050F4923009F406C1933009F4C1
:10F660006DC0913009F059C253C0913109F477C08F
:10F67000923108F0BBC0903109F04FC2F5C098310B
:10F6800009F487C0993150F4953109F4EFC09531F0
:10F6900008F4C6C1963109F040C2C2C19A3109F4DA
:10F6A0006CC09A3108F491C09B3109F45BC09D3164
:10F6B00009F033C29D81903359F48F81882311F46E
:10F6C0009EE11CC0813011F091E018C098E916C08D
:10F6D000892F807591F0903539F4E0E0F0E089E011
:10F6E0008093570094910AC0983539F4E3E0F0E034
:10F6F00089E080935700949101C090E01A821B82A8
:10F700008D818C831D829E831F8227E030E009C299
:10F710001A8288E08B8381E48C8386E58D8382E581
:10F720008E8389E48F8383E5888780E589878FE5E9
:10F730008A8782E38B872BE030E0F3C18A818139AD
:10F7400041F0823941F0803911F48FE005C080E04A
:10F7500003C082E001C08AE01A828B8344C0772410
:10F76000739482C08D81882311F48EE12CC0813086
:10F7700011F081E028C088E926C01A82E1E0F0E0BB
:10F7800089E08093570084918B831C8224E030E0D1
:10F79000C8C18B81803589F48C81883039F4E2E0EE
:10F7A000F0E089E08093570084910DC0E0E0F0E044
:10F7B00089E080935700849106C0E3E0F0E089E09F
:10F7C0008093570084911A82DFCF8D81836C99E0FA
:10F7D000E1E0F0E0082E90935700E89507B600FCB2
:10F7E000FDCF1A821B8223E030E09BC180EC8A832C
:10F7F000CE5CDE4F188219821A821B82C253D1401E
:10F800008EC18A8190E0A0E0B0E0582F44273327D2
:10F8100022278B8190E0A0E0B0E0DC0199278827C7
:10F82000282B392B4A2B5B2B8D8190E0A0E0B0E098
:10F83000282B392B4A2B5B2B8C8190E0A0E0B0E089
:10F84000BA2FA92F982F8827282B392B4A2B5B2BCF
:10F85000220F331F441F551FC05EDE4F288339839C
:10F860004A835B83C052D1401A8259C13A81C95C34
:10F87000DE4F3883C753D140CA5CDE4F1882C6536F
:10F88000D1408B81C82EDD24CA5CDE4F488159816E
:10F89000C653D140C42AD52A933109F082C0CE5C28
:10F8A000DE4F88819981AA81BB81C253D1408050AB
:10F8B000904CA340B04030F583E0CE5CDE4FE88052
:10F8C000F9800A811B81C253D140F70100935B008C
:10F8D00080935700E89507B600FCFDCFCE5CDE4F65
:10F8E000088119812A813B81C253D14000501F4FAA
:10F8F0002F4F3F4FCE5CDE4F088319832A833B8313
:10F90000C253D140C05EDE4F488159816A817B81FC
:10F91000C052D140DE011B9631E08C9111962C91A2
:10F9200011971296C75CDE4F2883C953D140C85C3B
:10F93000DE4F1882C853D14090E0C85CDE4FE881AA
:10F94000F981C853D1408E2B9F2B0C01FA01609393
:10F950005B0030935700E89511244E5F5F4F6F4F67
:10F960007F4F0EEFE02E0FEFF02ECE0CDF1CC114F8
:10F97000D10499F685E0C05EDE4F088119812A81A5
:10F980003B81C052D140F80120935B008093570027
:10F99000E89507B600FCFDCF81E180935700E8951C
:10F9A00035C0C05EDE4F88819981AA81BB81C0527B
:10F9B000D140B695A795979587957C018601ABE0D8
:10F9C000AA2EB12CAC0EBD1E0BC0D5016D915D01F0
:10F9D000C7010F947FFE0894E11CF11C01501040F8
:10F9E0000115110591F7A60160E070E0440F551F65
:10F9F000661F771FC05EDE4FE880F9800A811B8199
:10FA0000C052D1404E0D5F1D601F711F1A82C05E33
:10FA1000DE4F488359836A837B83C052D1407FC0C5
:10FA2000FA80C55CDE4FF882CB53D140C65CDE4F16
:10FA30001882CA53D1408B81C82EDD24C65CDE4FAC
:10FA400008811981CA53D140C02AD12A1A828981DA
:10FA5000BE016D5F7F4F843121F59601C05EDE4FA0
:10FA6000E880F9800A811B81C052D1400BBFF701A9
:10FA700087919691DB018C9311969C936E5F7F4FDB
:10FA8000D801C7010296A11DB11DC05EDE4F88835B
:10FA90009983AA83BB83C052D14022503040F1F6F3
:10FAA00036C0C05EDE4F288139814A815B81C052F9
:10FAB000D1400894C108D108760100E010E0089414
:10FAC000C11CD11C0894E11CF11C011D111DE20E8A
:10FAD000F31E041F151F21BDBB27A52F942F832FB5
:10FAE00082BD2F5F3F4F4F4F5F4FF89A80B5DB01CC
:10FAF0008D93BD012E153F054007510761F7C05E8C
:10FB0000DE4F288339834A835B83C052D1409601FC
:10FB10002D5F3F4FFB01108204C080EC8A8322E0FE
:10FB200030E08BE18093C6008091C00086FFFCCF5F
:10FB30008091C00080648093C000C15DDE4FF88179
:10FB4000CF52D140F093C6008091C00086FFFCCF19
:10FB50008091C00080648093C000432F3093C60022
:10FB60008091C00086FFFCCF8091C00080648093AC
:10FB7000C000922F2093C6008091C00086FFFCCF6A
:10FB80008091C00080648093C0008EE08093C600A6
:10FB90008091C00086FFFCCF8091C000806480937C
:10FBA000C00065E1C15DDE4FE880CF52D1406E25D7
:10FBB00069276427FE01319610C090819093C6009A
:10FBC0008091C00086FFFCCF31968091C000806498
:10FBD0008093C0006927215030402115310569F715
:10FBE0006093C6008091C00086FFFCCF8091C0006A
:10FBF00080648093C00085B1805885B9772081F4F6
:10FC0000C15DDE4F0881CF52D1400F5FC15DDE4F35
:10FC10000883CF52D14090E0A0E0B0E00D941AF4F8
:10FC200027982F9880E090E020ED37E0F901319798
:10FC3000F1F7019684369105C9F700008091C00064
:10FC40008D7F8093C00081E180935700E895EE2777
:10FC5000FF270994FFCF90E00D941AF497FB092E2B
:10FC600007260AD077FD04D02ED006D000201AF443
:10FC7000709561957F4F0895F6F7909581959F4F08
:10FC80000895A1E21A2EAA1BBB1BFD010DC0AA1FDD
:10FC9000BB1FEE1FFF1FA217B307E407F50720F0F5
:10FCA000A21BB30BE40BF50B661F771F881F991F70
:10FCB0001A9469F760957095809590959B01AC01B9
:10FCC000BD01CF010895AA1BBB1B51E107C0AA1FAC
:10FCD000BB1FA617B70710F0A61BB70B881F991FED
:10FCE0005A95A9F780959095BC01CD010895F99991
:10FCF000FECF92BD81BDF89A992780B50895262F31
:10FD0000F999FECF1FBA92BD81BD20BD0FB6F89400
:0EFD1000FA9AF99A0FBE01960895F894FFCF63
:040000033000E000E9
:00000001FF
